:020000040000FA
:0408000008EF0CF001
:1008100003B273EF05F0F2B491EF05F09EB099EFDB
:1008200005F09EB2A1EF05F0F2A81AEF04F0F2B2C3
:1008300021EF04F0F2B01FEF04F0B7EF0BF0F296E7
:10084000F290CD90F2929EA02BEF04F00101533F65
:100850002BEF04F0542BB2C1B6F1B3C1B7F1B4C160
:10086000B8F1B5C1B9F1AEC1B2F1AFC1B3F1B0C128
:10087000B4F1B1C1B5F1AAC1AEF1ABC1AFF1ACC138
:10088000B0F1ADC1B1F1A6C1AAF1A7C1ABF1A8C148
:10089000ACF1A9C1ADF1A2C1A6F1A3C1A7F1A4C158
:1008A000A8F1A5C1A9F19EC1A2F19FC1A3F1A0C168
:1008B000A4F1A1C1A5F19AC19EF19BC19FF19CC178
:1008C000A0F19DC1A1F1CECF9AF1CFCF9BF153C141
:1008D0009CF154C19DF1CF6ACE6A0101536B546BF8
:1008E0009E90CD800FBC0F8E0FBA7AEF04F00F8A66
:1008F000B7EF0BF013880F8C0FBEB7EF04F09AC15F
:100900009EF19BC19FF19CC1A0F19DC1A1F19EC12F
:10091000A2F19FC1A3F1A0C1A4F1A1C1A5F1A2C1FF
:10092000A6F1A3C1A7F1A4C1A8F1A5C1A9F1A6C1CF
:10093000AAF1A7C1ABF1A8C1ACF1A9C1ADF1AAC19F
:10094000AEF1ABC1AFF1ACC1B0F1ADC1B1F1AEC16F
:10095000B2F1AFC1B3F1B0C1B4F1B1C1B5F1B2C13F
:10096000B6F1B3C1B7F1B4C1B8F1B5C1B9F1010184
:100970005E6B5F6B606B616B9A515E279B515F236F
:100980009C5160239D5161239E515E279F515F239F
:10099000A0516023A1516123A2515E27A3515F237F
:1009A000A4516023A5516123A6515E27A7515F235F
:1009B000A8516023A9516123AA515E27AB515F233F
:1009C000AC516023AD516123AE515E27AF515F231F
:1009D000B0516023B1516123B2515E27B3515F23FF
:1009E000B4516023B5516123B6515E27B7515F23DF
:1009F000B8516023B9516123D8900101613360334C
:100A00005F335E33D8900101613360335F335E330F
:100A1000D8900101613360335F335E3300C10CF164
:100A200001C10DF102C10EF103C10FF104C110F1BA
:100A300005C111F106C112F107C113F108C114F18A
:100A400009C115F10AC116F10BC117F134C135F115
:100A500011B836EF05F00101620E046F010E056F4B
:100A6000000E066F000E076F3FEF05F00101A70EA5
:100A7000046F020E056F000E066F000E076F5EC159
:100A800000F15FC101F160C102F161C103F14AEC03
:100A900037F003BF04D019BE02D019A0108C11A0EA
:100AA00057EF05F010BA57EF05F00F80108A0CC110
:100AB00000F10DC101F10EC102F10FC103F110C12E
:100AC00004F111C105F112C106F113C107F114C1FE
:100AD00008F115C109F116C10AF117C10BF135C1B1
:100AE00034F1B7EF0BF00392ABB2AB98AB880301D4
:100AF00003EE00F080517F0BE92604C0EFFF802B4E
:100B00008151805D700BD8A48B8200008051815D83
:100B1000700BD8A48B9281518019D8B40790B7EF8D
:100B20000BF0F2940101453FB7EF0BF0462BB7EF06
:100B30000BF09E900101533FB7EF0BF0542BB7EF32
:100B40000BF09E9211B87DEF08F0040066A1A9EFAA
:100B500005F08BB4B3EF05F010ACB3EF05F08B8468
:100B6000109CB4EF05F08B9407B406EF06F007B0C5
:100B700006EF06F01EC620F61FC621F61CC61EF69E
:100B80001DC61FF61AC61CF61BC61DF606C608F6BD
:100B900007C609F604C606F605C607F602C604F639
:100BA00003C605F626C628F627C629F624C626F665
:100BB00025C627F622C624F623C625F60EC610F64D
:100BC0000FC611F60CC60EF60DC60FF60AC60CF6C9
:100BD0000BC60DF62EC630F62FC631F62CC62EF6F5
:100BE0002DC62FF62AC62CF62BC62DF616C618F6DD
:100BF00017C619F614C616F615C617F612C614F659
:100C000013C615F62BEC39F0D9EC38F0077C07AC9D
:100C100021EF06F0C274C2B41BEF06F0C3CFB7F5E4
:100C2000C4CFB8F50501D890B833B733D890B833EE
:100C3000B73322EF06F0C3CF55F1C4CF56F122EF00
:100C400006F0C28207B494EF06F047C14BF148C1E9
:100C50004CF149C14DF14AC14EF15EC162F15FC133
:100C600063F160C164F161C165F113A83AEF06F068
:100C7000138C13989AC1BAF19BC1BBF19CC1BCF112
:100C80009DC1BDF19EC1BEF19FC1BFF1A0C1C0F128
:100C9000A1C1C1F1A2C1C2F1A3C1C3F1A4C1C4F1F8
:100CA000A5C1C5F1A6C1C6F1A7C1C7F1A8C1C8F1C8
:100CB000A9C1C9F1AAC1CAF1ABC1CBF1ACC1CCF198
:100CC000ADC1CDF1AEC1CEF1AFC1CFF1B0C1D0F168
:100CD000B1C1D1F1B2C1D2F1B3C1D3F1B4C1D4F138
:100CE000B5C1D5F1B6C1D6F1B7C1D7F1B8C1D8F108
:100CF000B9C1D9F1B7C5B9F5B8C5BAF5B9C5BBF52C
:100D0000BAC5BCF5010155515B2756515C23E86A11
:100D10005D230E2E94EF06F05CC157F15DC158F1D2
:100D20005B6B5C6B5D6B078E0201002FB7EF0BF006
:100D30003C0E006F1A50E00BE00AE866128818BEFD
:100D400002D018B4108E00C10CF101C10DF102C126
:100D50000EF103C10FF104C110F105C111F106C17B
:100D600012F107C113F108C114F109C115F10AC14B
:100D700016F10BC117F134C135F181AA75EF07F0F7
:100D800030A045EF07F005012F51000AD8B475EFE8
:100D900007F005012F51010AD8B4FEEF06F0050156
:100DA0002F51020AD8B43FEF07F005012F51030A73
:100DB000D8B43FEF07F005012F51040AD8B43FEF34
:100DC00007F005012F51050AD8B43FEF07F00501E0
:100DD0002F51060AD8B43FEF07F005012F51070A3B
:100DE000D8B43FEF07F005012F51320AD8B4FCEF19
:100DF00006F02F6B75EF07F075EF07F005015767E9
:100E000009EF07F0586709EF07F0596709EF07F096
:100E10005A670DEF07F075EF07F05BC500F15CC591
:100E200001F15DC502F15EC503F10101010E046F20
:100E3000000E056F000E066F000E076F4AEC37F0CC
:100E400000C15BF501C15CF502C15DF503C15EF552
:100E5000006732EF07F0016732EF07F0026732EF09
:100E600007F0036775EF07F057C55BF558C55CF5EC
:100E700059C55DF55AC55EF50F8875EF07F0050198
:100E8000306745EF07F075EF07F00FBE5AEF07F038
:100E900010A05FEF07F00101476756EF07F04867C2
:100EA00056EF07F0496756EF07F04A675AEF07F029
:100EB0005FEF07F007AE5FEF07F072EF07F0050195
:100EC000312F75EF07F03C0E316F302F75EF07F0C3
:100ED0000101000E626FE00E636FA50E646F010EDC
:100EE000656F13880501306B0F880501666B37B796
:100EF0007BEF07F066810CC100F10DC101F10EC15D
:100F000002F10FC103F110C104F111C105F112C1C9
:100F100006F113C107F114C108F115C109F116C199
:100F20000AF117C10BF135C134F100C10CF101C157
:100F30000DF102C10EF103C10FF104C110F105C1A1
:100F400011F106C112F107C113F108C114F109C171
:100F500015F10AC116F10BC117F134C135F10101C8
:100F60008E67BAEF07F08F67BAEF07F09067BAEFB6
:100F700007F09167BEEF07F0EEEF07F092C100F1C6
:100F800093C101F194C102F195C103F10101010E78
:100F9000046F000E056F000E066F000E076F4AEC1F
:100FA00037F000C192F101C193F102C194F103C184
:100FB00095F10067E3EF07F00167E3EF07F00267E1
:100FC000E3EF07F00367EEEF07F08EC192F18FC1F8
:100FD00093F190C194F191C195F10F80D57ED5BE6A
:100FE0006ED0D6CF47F1D7CF48F145C149F1E86A75
:100FF000E8CF4AF1138A19BE02D019A0108C1090C4
:1010000047C100F148C101F149C102F14AC103F1F0
:1010100001010A0E046F000E056F000E066F000E30
:10102000076F4AEC37F003AF1080010154A725EF9A
:1010300008F00F9A0F9C0F9E0101000E5E6F600E6C
:101040005F6F3D0E606F080E616F010147BF35EFA6
:1010500008F0486735EF08F0496735EF08F04A6750
:1010600035EF08F0F2885AEF08F0F2985E6B5F6B8C
:10107000606B616B9A6B9B6B9C6B9D6B9E6B9F6BAC
:10108000A06BA16BA26BA36BA46BA56BA66BA76BEC
:10109000A86BA96BAA6BAB6BAC6BAD6BAE6BAF6B9C
:1010A000B06BB16BB26BB36BB46BB56BB66BB76B4C
:1010B000B86BB96BD76AD66A0101456B466B0CC138
:1010C00000F10DC101F10EC102F10FC103F110C118
:1010D00004F111C105F112C106F113C107F114C1E8
:1010E00008F115C109F116C10AF117C10BF135C19B
:1010F00034F1B7EF0BF0B7EF0BF00201002FC9EF9F
:101100000AF0D59ED6CF47F1D7CF48F145C149F176
:10111000E86AE8CF4AF1138AD76AD66A0101456BBB
:10112000466BD58E1A50E00BE00AE866128818BEAE
:1011300002D018B4108E17AE1C8C00C10CF101C186
:101140000DF102C10EF103C10FF104C110F105C18F
:1011500011F106C112F107C113F108C114F109C15F
:1011600015F10AC116F10BC117F134C135F10FA009
:10117000109A11B8C7EF08F00101620E046F010E5A
:10118000056F000E066F000E076FD0EF08F001012B
:10119000A70E046F020E056F000E066F000E076F9C
:1011A00047C100F148C101F149C102F14AC103F14F
:1011B0004AEC37F003BFE3EF08F019BE02D019A0E4
:1011C000108C11B00F800CC100F10DC101F10EC1E6
:1011D00002F10FC103F110C104F111C105F112C1F7
:1011E00006F113C107F114C108F115C109F116C1C7
:1011F0000AF117C10BF135C134F102013C0E006F49
:1012000000C10CF101C10DF102C10EF103C10FF1DA
:1012100004C110F105C111F106C112F107C113F1AA
:1012200008C114F109C115F10AC116F10BC117F17A
:1012300034C135F181AAD2EF09F030A0A2EF09F054
:1012400005012F51000AD8B4D2EF09F005012F5142
:10125000010AD8B45BEF09F005012F51020AD8B496
:101260009CEF09F005012F51030AD8B49CEF09F057
:1012700005012F51040AD8B49CEF09F005012F5144
:10128000050AD8B49CEF09F005012F51060AD8B41D
:101290009CEF09F005012F51070AD8B49CEF09F023
:1012A00005012F51320AD8B459EF09F02F6BD2EF54
:1012B00009F0D2EF09F00501576766EF09F05867AA
:1012C00066EF09F0596766EF09F05A676AEF09F0AF
:1012D000D2EF09F05BC500F15CC501F15DC502F11B
:1012E0005EC503F10101010E046F000E056F000ED3
:1012F000066F000E076F4AEC37F000C15BF501C1C5
:101300005CF502C15DF503C15EF500678FEF09F082
:1013100001678FEF09F002678FEF09F00367D2EFE3
:1013200009F057C55BF558C55CF559C55DF55AC55B
:101330005EF50F88D2EF09F005013067A2EF09F0E2
:10134000D2EF09F00FBEB7EF09F010A0BCEF09F023
:1013500001014767B3EF09F04867B3EF09F0496748
:10136000B3EF09F04A67B7EF09F0BCEF09F007AE39
:10137000BCEF09F0CFEF09F00501312FD2EF09F0F2
:101380003C0E316F302FD2EF09F00101000E626F79
:10139000E00E636FA50E646F010E656F1388050183
:1013A000306B0F880501666B37B7D8EF09F066819F
:1013B0000CC100F10DC101F10EC102F10FC103F129
:1013C00010C104F111C105F112C106F113C107F1F9
:1013D00014C108F115C109F116C10AF117C10BF1C9
:1013E00035C134F100C10CF101C10DF102C10EF1A2
:1013F00003C10FF104C110F105C111F106C112F1D1
:1014000007C113F108C114F109C115F10AC116F1A0
:101410000BC117F134C135F101018E6717EF0AF0E6
:101420008F6717EF0AF0906717EF0AF091671BEFCD
:101430000AF04BEF0AF092C100F193C101F194C19F
:1014400002F195C103F10101010E046F000E056F59
:10145000000E066F000E076F4AEC37F000C192F1E4
:1014600001C193F102C194F103C195F1006740EF0E
:101470000AF0016740EF0AF0026740EF0AF00367E5
:101480004BEF0AF08EC192F18FC193F190C194F1AC
:1014900091C195F10F80109047C100F148C101F151
:1014A00049C102F14AC103F101010A0E046F000EA5
:1014B000056F000E066F000E076F4AEC37F003AFA2
:1014C0001080010154A771EF0AF00F9A0F9C0F9E34
:1014D0000101000E5E6F600E5F6F3D0E606F080EC3
:1014E000616F47C100F148C101F149C102F14AC130
:1014F00003F10101140E046F050E056F000E066F57
:10150000000E076F4AEC37F003AF8AEF0AF0F2885B
:10151000AFEF0AF0F2985E6B5F6B606B616B9A6B7A
:101520009B6B9C6B9D6B9E6B9F6BA06BA16BA26B6F
:10153000A36BA46BA56BA66BA76BA86BA96BAA6B1F
:10154000AB6BAC6BAD6BAE6BAF6BB06BB16BB26BCF
:10155000B36BB46BB56BB66BB76BB86BB96B0CC1D7
:1015600000F10DC101F10EC102F10FC103F110C173
:1015700004F111C105F112C106F113C107F114C143
:1015800008F115C109F116C10AF117C10BF135C1F6
:1015900034F104008BB4D4EF0AF010ACD4EF0AF0AD
:1015A0008B84109CD5EF0AF08B9407B427EF0BF0D7
:1015B00007B027EF0BF01EC620F61FC621F61CC68B
:1015C0001EF61DC61FF61AC61CF61BC61DF606C65D
:1015D00008F607C609F604C606F605C607F602C6EB
:1015E00004F603C605F626C628F627C629F624C63D
:1015F00026F625C627F622C624F623C625F60EC6ED
:1016000010F60FC611F60CC60EF60DC60FF60AC67A
:101610000CF60BC60DF62EC630F62FC631F62CC6CC
:101620002EF62DC62FF62AC62CF62BC62DF616C67C
:1016300018F617C619F614C616F615C617F612C60A
:1016400014F613C615F62BEC39F0D9EC38F0077CFC
:1016500007AC42EF0BF0C274C2B43CEF0BF0C3CF47
:10166000B7F5C4CFB8F50501D890B833B733D890E3
:10167000B833B73343EF0BF0C3CF55F1C4CF56F1B6
:1016800043EF0BF0C28207B4B5EF0BF047C14BF14B
:1016900048C14CF149C14DF14AC14EF15EC162F100
:1016A0005FC163F160C164F161C165F113A85BEFD3
:1016B0000BF0138C13989AC1BAF19BC1BBF19CC17A
:1016C000BCF19DC1BDF19EC1BEF19FC1BFF1A0C1E2
:1016D000C0F1A1C1C1F1A2C1C2F1A3C1C3F1A4C1B2
:1016E000C4F1A5C1C5F1A6C1C6F1A7C1C7F1A8C182
:1016F000C8F1A9C1C9F1AAC1CAF1ABC1CBF1ACC152
:10170000CCF1ADC1CDF1AEC1CEF1AFC1CFF1B0C121
:10171000D0F1B1C1D1F1B2C1D2F1B3C1D3F1B4C1F1
:10172000D4F1B5C1D5F1B6C1D6F1B7C1D7F1B8C1C1
:10173000D8F1B9C1D9F1B7C5B9F5B8C5BAF5B9C5C8
:10174000BBF5BAC5BCF5010155515B2756515C2369
:10175000E86A5D230E2EB5EF0BF05CC157F15DC159
:1017600058F15B6B5C6B5D6B078EB7EF0BF002C0E3
:10177000E0FF005001C0D8FF1000A6B2BDEF0BF093
:101780000CC0A9FF0BC0A8FFA69EA69CA684F29E33
:10179000550EA76EAA0EA76EA682F28EA694A6B2CA
:1017A000CFEF0BF00C2A1200A96EA69EA69CA68075
:1017B000A8500C2A120004012C0E826F5CEC0FF072
:1017C00045EC38F00C50D4EC0BF0E8CF00F10C50A5
:1017D000D4EC0BF0E8CF01F101AFF4EF0BF0010115
:1017E000FF0E026FFF0E036FE8EC37F0296700EF82
:1017F0000CF00401200E826F5CEC0FF005EF0CF092
:1018000004012D0E826F5CEC0FF0F2EC35F012004B
:10181000306A076A0F6A106A116A126A136A0F0146
:101820000D0EC16E860EC06E030EC26E0F01680EE5
:10183000896E130E926E080E8A6E8A6AF30E936E8C
:101840008B6A900E946EC80ED4EC0BF0E8CFE8FFD4
:101850001098E8A0108810A805D00E0E226E8E0EEB
:10186000236E04D00F0E226E8F0E236EE3EC39F040
:10187000F18EF19EFC0ED4EC0BF0E8CF0BF00BA038
:1018800011800BA211820BA411840BA81188C90E20
:10189000D4EC0BF0E8CF17F0CA0ED4EC0BF0E8CF85
:1018A00018F0CB0ED4EC0BF0E8CF19F0CC0ED4EC42
:1018B0000BF0E8CF1AF0CD0ED4EC0BF0E8CF2FF000
:1018C0001C6A1D6A0E6A01015B6B5C6B5D6B576B7A
:1018D000586BF29A0101476B486B496B4A6B4B6B33
:1018E0004C6B4D6B4E6B4F6B506B516B526B456B32
:1018F000466BD76AD66A0F01280ED56EF28A9D9084
:10190000B00ECD6E01015E6B5F6B606B616B626BE5
:10191000636B646B656B666B676B686B696B536B52
:10192000546BCF6ACE6A0F9A0F9C0F9E9D80760EE5
:10193000CA6E9D8202013C0E006FCC6A160ED4EC7A
:101940000BF0E8CF00F1170ED4EC0BF0E8CF01F16B
:10195000180ED4EC0BF0E8CF02F1190ED4EC0BF01A
:10196000E8CF03F1010103AFD0EF0CF045EC38F004
:10197000160E0C6E00C10BF0BDEC0BF0170E0C6ECA
:1019800001C10BF0BDEC0BF0180E0C6E02C10BF098
:10199000BDEC0BF0190E0C6E03C10BF0BDEC0BF09F
:1019A00000C18EF101C18FF102C190F103C191F12B
:1019B00000C192F101C193F102C194F103C195F10B
:1019C0001A0ED4EC0BF0E8CF00F11B0ED4EC0BF0A8
:1019D000E8CF01F11C0ED4EC0BF0E8CF02F11D0EA4
:1019E000D4EC0BF0E8CF03F1010103AF26EF0DF0CB
:1019F00045EC38F01A0E0C6E00C10BF0BDEC0BF08C
:101A00001B0E0C6E01C10BF0BDEC0BF01C0E0C6E2E
:101A100002C10BF0BDEC0BF01D0E0C6E03C10BF000
:101A2000BDEC0BF01A0ED4EC0BF0E8CF00F11B0E5E
:101A3000D4EC0BF0E8CF01F11C0ED4EC0BF0E8CFA6
:101A400002F11D0ED4EC0BF0E8CF03F100C196F1CA
:101A500001C197F102C198F103C199F1240EAC6E56
:101A6000900EAB6E240EAC6E080EB86E000EB06E0B
:101A70001F0EAF6E0401806B816B0F01900EAB6E79
:101A80000F019D8A0301806B816BC26B8B9287EC87
:101A90003EF087EC3EF0880ED4EC0BF0E8CF00F17E
:101AA000890ED4EC0BF0E8CF01F1010101AF71EF29
:101AB0000DF045EC38F0880E0C6E00C10BF0BDEC5B
:101AC0000BF0890E0C6E01C10BF0BDEC0BF0880E13
:101AD000D4EC0BF0E8CF00F1890ED4EC0BF0E8CF9A
:101AE00001F100C140F601C141F602C142F603C155
:101AF00043F6E1EC41F066EC3CF0200ED4EC0BF048
:101B0000E8CF2FF505012F51FF0AD8A48FEF0DF074
:101B10002F6B200E0C6E2FC50BF0BDEC0BF00501EA
:101B2000010E306F3C0E316F250ED4EC0BF0E8CF78
:101B300000F1260ED4EC0BF0E8CF01F1270ED4EC27
:101B40000BF0E8CF02F1280ED4EC0BF0E8CF03F154
:101B5000010103AFC6EF0DF045EC38F0250E0C6E19
:101B600000C10BF0BDEC0BF0260E0C6E01C10BF0AA
:101B7000BDEC0BF0270E0C6E02C10BF0BDEC0BF0B0
:101B8000280E0C6E03C10BF0BDEC0BF000C157F535
:101B900001C158F502C159F503C15AF500C15BF501
:101BA00001C15CF502C15DF503C15EF5290ED4ECFF
:101BB0000BF0E8CF5FF5050160515F5DD8A05FC510
:101BC00060F5210ED4EC0BF0E8CF00F1220ED4EC3E
:101BD0000BF0E8CF01F1230ED4EC0BF0E8CF02F1CB
:101BE000240ED4EC0BF0E8CF03F1010103AF27EF93
:101BF0000EF045EC38F0210E0C6E00C10BF0BDEC80
:101C00000BF0220E0C6E01C10BF0BDEC0BF0230E9D
:101C10000C6E02C10BF0BDEC0BF0240E0C6E03C178
:101C20000BF0BDEC0BF0210ED4EC0BF0E8CF00F183
:101C3000220ED4EC0BF0E8CF01F1230ED4EC0BF024
:101C4000E8CF02F1240ED4EC0BF0E8CF03F100C191
:101C500061F501C162F502C163F503C164F5AEEC43
:101C60003BF094EC3AF0ECEC39F030A098EF0EF049
:101C700005012F51020A16E005012F51030A19E050
:101C800005012F51040A24E005012F51050A2BE01C
:101C900005012F51060A39E005012F51070A3FE0DF
:101CA00098EF0EF0602F95EF0EF05FC560F598EF9E
:101CB0000EF0B0C500F101010F0E00170101005137
:101CC000000A36E001010051050A32E095EF0EF0FE
:101CD000B0C500F101010F0E001701010051000A0B
:101CE00027E095EF0EF00501B051000A21E0050153
:101CF000B051150A1DE00501B051300A19E0050187
:101D0000B051450A15E095EF0EF00501B051000AFB
:101D10000FE00501B051300A0BE095EF0EF0050120
:101D2000B051000A05E095EF0EF081BA20EF42F0C5
:101D30007DEC39F007900001F28EF28C12AE03D0E8
:101D400012BC6FEF20F007B08BEF33F00FB09EEFB7
:101D50002CF010BE9EEF2CF012B89EEF2CF00FB8B6
:101D60002CEF26F00301805181197F0BD8B48BEF43
:101D700033F013EE00F081517F0BE126812BE7CF8A
:101D8000E8FFE00BD8B48BEF33F023EE82F0C251C2
:101D90003F0BD926E7CFDFFFC22BDF50780AD8A44C
:101DA0008BEF33F0078092C100F193C101F194C130
:101DB00002F195C103F10101040E046F000E056FDD
:101DC000000E066F000E076F4AEC37F000AFF2EF1F
:101DD0000EF00101030E926F000E936F000E946FD0
:101DE000000E956F03018251720AD8B47AEF2CF07D
:101DF0008251520AD8B47AEF2CF08251750AD8B4C5
:101E00007AEF2CF08251630AD8B445EF30F082515A
:101E1000690AD8B424EF29F082517A0AD8B437EF8E
:101E20002AF08251490AD8B4C3EF28F08251500AEF
:101E3000D8B4E1EF27F08251700AD8B424EF28F02B
:101E40008251540AD8B44FEF28F08251740AD8B4A2
:101E500095EF28F08251410AD8B472EF10F0825108
:101E60004B0AD8B470EF0FF082516D0AD8B4A5EFC9
:101E700014F082514D0AD8B4BEEF14F08251730AA7
:101E8000D8B4AAEF2BF08251530AD8B40FEF2CF03C
:101E900082514C0AD8B421EF1CF08251760AD8B492
:101EA0004DEF15F08251590AD8B4F6EF13F012AE87
:101EB00001D0128C7CEF30F0040114EE00F0805160
:101EC0007F0BE12682C4E7FF802B120004010D0E78
:101ED000826F5CEC0FF00A0E826F5CEC0FF0120068
:101EE00004014B0E826F5CEC0FF004012C0E826F2C
:101EF0005CEC0FF081B802D02FB630D003018351D3
:101F0000430AD8B4B5EF0FF003018351630AD8B484
:101F1000B7EF0FF003018351520AD8B4B9EF0FF0B5
:101F200003018351720AD8B4BBEF0FF00301835150
:101F3000470AD8B4BDEF0FF003018351670AD8B444
:101F4000BFEF0FF003018351540AD8B4C1EF0FF073
:101F500003018351740AD8B430EF10F003018351A8
:101F6000550AD8B4C3EF0FF082D02F807AD02F90CB
:101F700078D02F8276D02F9274D02F8472D02F9465
:101F800070D02F866ED084C330F185C331F186C303
:101F900032F187C333F10101296B93EC38F00AEC7D
:101FA00038F000C104F101C105F102C106F103C11D
:101FB00007F186EC38F0200EF86EF76AF66A090031
:101FC000F5CF2CF10900F5CF2DF10900F5CF2EF159
:101FD0000900F5CF2FF10900F5CF30F10900F5CF59
:101FE00031F10900F5CF32F10900F5CF33F10101EC
:101FF000296B93EC38F00AEC38F04AEC37F00067C4
:1020000009EF10F0016709EF10F0026709EF10F017
:10201000036701D025D004014E0E826F5CEC0FF0F7
:1020200004016F0E826F5CEC0FF004014D0E826FA5
:102030005CEC0FF00401610E826F5CEC0FF00401A8
:10204000740E826F5CEC0FF00401630E826F5CEC27
:102050000FF00401680E826F5CEC0FF07AEF30F045
:102060002F96CD0E0C6E2FC00BF0BDEC0BF0CD0EED
:10207000D4EC0BF0E8CF2FF02FB006D00401630EA4
:10208000826F5CEC0FF005D00401430E826F5CECB4
:102090000FF02FB206D00401720E826F5CEC0FF0CD
:1020A00005D00401520E826F5CEC0FF02FB406D005
:1020B0000401670E826F5CEC0FF005D00401470E3F
:1020C000826F5CEC0FF02FB606D00401740E826FA5
:1020D0005CEC0FF005D00401540E826F5CEC0FF045
:1020E0007AEF30F00401410E826F5CEC0FF00301D7
:1020F0008351310AD8B416EF13F003018351320A29
:10210000D8B446EF12F003018351330AD8B4CFEFAD
:1021100011F003018351340AD8B4BFEF10F003016A
:102120008351350AD8B49CEF10F004013F0E826F42
:102130005CEC0FF07AEF30F004012C0E826F5CEC57
:102140000FF003018451300AD8B4AFEF10F003014F
:102150008451310AD8B4B7EF10F008EF12F08B9029
:102160000401300E826F5CEC0FF0BDEF10F08B803D
:102170000401310E826F5CEC0FF07AEF30F0CC0E80
:10218000D4EC0BF0E8CF0BF004012C0E826F5CEC6A
:102190000FF003018451310AD8B4E3EF10F00301CA
:1021A0008451300AD8B4E5EF10F0030184514D0A90
:1021B000D8B4EFEF10F003018451540AD8B4F6EF0D
:1021C00010F00DEF11F08A8401D08A940BAE04D088
:1021D0000BAC02D00BBA21D0E00E0B1218D01F0EA0
:1021E0000B168539E844E00B0B1211D0E00E0B16EC
:1021F00086EC38F085C332F186C333F10101296BD7
:1022000093EC38F00AEC38F000511F0B0B12CC0E97
:102210000C6E0BC00BF0BDEC0BF00401340E826FA2
:102220005CEC0FF004012C0E826F5CEC0FF0CC0E16
:10223000D4EC0BF0E8CF1AF08AB406D00401300ECB
:10224000826F5CEC0FF005D00401310E826F5CEC04
:102250000FF004012C0E826F5CEC0FF01A38E8408E
:10226000070BE8CF82F40401300E82275CEC0FF0FC
:1022700004012C0E826F5CEC0FF045EC38F01A5024
:102280001F0BE8CF00F1E8EC37F032C182F4040113
:10229000300E82275CEC0FF033C182F40401300E63
:1022A00082275CEC0FF004012C0E826F5CEC0FF0C7
:1022B00045EC38F02DC000F100AF0BD0FF0E016FE0
:1022C000FF0E026FFF0E036F04012D0E826F5CEC98
:1022D0000FF0E8EC37F031C182F40401300E8227B0
:1022E0005CEC0FF032C182F40401300E82275CEC0A
:1022F0000FF033C182F40401300E82275CEC0FF042
:1023000004012C0E826F5CEC0FF045EC38F02CC011
:1023100000F1E8EC37F031C182F40401300E82277D
:102320005CEC0FF032C182F40401300E82275CECC9
:102330000FF033C182F40401300E82275CEC0FF001
:1023400004012C0E826F5CEC0FF045EC38F02EC0CF
:1023500000F100AF0BD0FF0E016FFF0E026FFF0EFA
:10236000036F04012D0E826F5CEC0FF0E8EC37F088
:1023700031C182F40401300E82275CEC0FF032C1CF
:1023800082F40401300E82275CEC0FF033C182F43A
:102390000401300E82275CEC0FF07AEF30F0CB0EA8
:1023A000D4EC0BF0E8CF0BF004012C0E826F5CEC48
:1023B0000FF003018451450AD8B4F3EF11F0030183
:1023C0008451440AD8B4F6EF11F003018451300A65
:1023D000D8B4F9EF11F003018451310AD8B4FDEFFC
:1023E00011F008EF12F00B9E02EF12F00B8E02EFCD
:1023F00012F0FC0E0B1602EF12F0FC0E0B160B8007
:1024000002EF12F0CB0E0C6E0BC00BF0BDEC0BF01C
:102410000401330E826F5CEC0FF004012C0E826F0E
:102420005CEC0FF0CB0ED4EC0BF0E8CF19F019BE3A
:1024300021EF12F00401450E826F5CEC0FF026EFE5
:1024400012F00401440E826F5CEC0FF004012C0EBC
:10245000826F5CEC0FF00401300E826F5CEC0FF0C9
:1024600004012C0E826F5CEC0FF019B03FEF12F0FC
:102470000401300E826F5CEC0FF044EF12F00401A7
:10248000310E826F5CEC0FF07AEF30F0CA0ED4ECB4
:102490000BF0E8CF0BF004012C0E826F5CEC0FF018
:1024A00003018451450AD8B482EF12F0030184512C
:1024B000440AD8B485EF12F0030184514D0AD8B410
:1024C0008EEF12F003018451410AD8B488EF12F064
:1024D00003018451460AD8B48BEF12F003018451F2
:1024E000560AD8B496EF12F003018451500AD8B4BA
:1024F000A1EF12F003018451520AD8B4A4EF12F0F4
:10250000ADEF12F00B9EA7EF12F00B8EA7EF12F0BB
:102510000B9CA7EF12F00B8CA7EF12F0FC0E0B1622
:1025200085C3E8FF030B0B12A7EF12F0C70E0B16C3
:1025300085C3E8FF070BE846E846E8460B12A7EF1D
:1025400012F00B84A7EF12F00B94A7EF12F0CA0E53
:102550000C6E0BC00BF0BDEC0BF0CA0ED4EC0BF004
:10256000E8CF18F00401320E826F5CEC0FF004012A
:102570002C0E826F5CEC0FF018BEC6EF12F0040157
:10258000450E826F5CEC0FF0CBEF12F00401440EAD
:10259000826F5CEC0FF004012C0E826F5CEC0FF08C
:1025A00018C0E8FF030BE8CF82F40401300E822745
:1025B0005CEC0FF004012C0E826F5CEC0FF018BC89
:1025C000E9EF12F00401410E826F5CEC0FF0EEEFC8
:1025D00012F00401460E826F5CEC0FF004012C0E29
:1025E000826F5CEC0FF018C0E8FF380BE842E8425D
:1025F000E842E8CF82F40401300E82275CEC0FF051
:1026000004012C0E826F5CEC0FF018B40FEF13F086
:102610000401520E826F5CEC0FF014EF13F0040112
:10262000500E826F5CEC0FF07AEF30F0C90ED4ECF4
:102630000BF0E8CF0BF004012C0E826F5CEC0FF076
:1026400003018451450AD8B434EF13F003018451D7
:10265000440AD8B437EF13F0030184514D0AD8B4BB
:102660003AEF13F048EF13F00B9E42EF13F00B8E8E
:1026700042EF13F0F80E0B1685C3E8FF070B0B12A1
:1026800042EF13F0C90E0C6E0BC00BF0BDEC0BF05B
:102690000401310E826F5CEC0FF004012C0E826F8E
:1026A0005CEC0FF0C90ED4EC0BF0E8CF17F017BEBE
:1026B00006D00401450E826F5CEC0FF005D00401DA
:1026C000440E826F5CEC0FF004012C0E826F5CEC08
:1026D0000FF017C0E8FF070BE8CF82F40401300EBB
:1026E00082275CEC0FF004012C0E826F5CEC0FF083
:1026F000078045EC38F028C0E8FF003B004300436A
:10270000030BE8EC37F033C182F40401300E82276A
:102710005CEC0FF004012C0E826F5CEC0FF045ECCA
:1027200038F028C001F1019F019D29C000F101018D
:10273000E8EC37F02FC182F40401300E82275CEC04
:102740000FF030C182F40401300E82275CEC0FF0F0
:1027500031C182F40401300E82275CEC0FF032C1EB
:1027600082F40401300E82275CEC0FF033C182F456
:102770000401300E82275CEC0FF004012C0E826FF6
:102780005CEC0FF045EC38F02AC001F12BC000F1F1
:10279000D89001330033D890013300330101E8ECC5
:1027A00037F02FC182F40401300E82275CEC0FF069
:1027B00030C182F40401300E82275CEC0FF031C18D
:1027C00082F40401300E82275CEC0FF032C182F4F7
:1027D0000401300E82275CEC0FF033C182F4040157
:1027E000300E82275CEC0FF07AEF30F0FC0ED4EC68
:1027F0000BF0E8CF0BF003018351520AD8B42DEF50
:1028000014F003018351720AD8B430EF14F00301BD
:102810008351500AD8B433EF14F003018351700A86
:10282000D8B436EF14F003018351550AD8B439EF08
:1028300014F003018351750AD8B43CEF14F003017E
:102840008351430AD8B445EF14F003018351630A5E
:10285000D8B448EF14F051EF14F00B904BEF14F094
:102860000B804BEF14F00B924BEF14F00B824BEFFD
:1028700014F00B944BEF14F00B844BEF14F00B9609
:102880004BEF14F00B864BEF14F00B984BEF14F05A
:102890000B884BEF14F0FC0E0C6E0BC00BF0BDEC74
:1028A0000BF00401590E826F5CEC0FF01190119245
:1028B00011941198FC0ED4EC0BF0E8CF0BF00BA0A8
:1028C00011800BA211820BA411840BA8118811A0F6
:1028D00071EF14F00401520E826F5CEC0FF076EF92
:1028E00014F00401720E826F5CEC0FF011A880EFFF
:1028F00014F00401430E826F5CEC0FF085EF14F0CE
:102900000401630E826F5CEC0FF011A28FEF14F0E4
:102910000401500E826F5CEC0FF094EF14F0040190
:10292000700E826F5CEC0FF011A49EEF14F00401A6
:10293000550E826F5CEC0FF0A3EF14F00401750EDE
:10294000826F5CEC0FF07AEF30F004016D0E826F55
:102950005CEC0FF003018351300AD8B4FDEF14F0A2
:1029600003018351310AD8B410EF15F003018351EC
:10297000320AD8B423EF15F07CEF30F004014D0E8D
:10298000826F5CEC0FF086EC38F084C331F185C3C4
:1029900032F186C333F10101296B93EC38F00AEC74
:1029A00038F003018351300AD8B4E5EF14F0030185
:1029B0008351310AD8B4EDEF14F003018351320A88
:1029C000D8B4F5EF14F07CEF30F0FD0E0C6E00C1C2
:1029D0000BF0BDEC0BF0FDEF14F0FE0E0C6E00C121
:1029E0000BF0BDEC0BF010EF15F0FF0E0C6E00C1FC
:1029F0000BF0BDEC0BF023EF15F00401300E826FED
:102A00005CEC0FF004012C0E826F5CEC0FF045ECD7
:102A100038F0FD0ED4EC0BF0E8CF00F134EF15F0F8
:102A20000401310E826F5CEC0FF004012C0E826FFA
:102A30005CEC0FF045EC38F0FE0ED4EC0BF0E8CF78
:102A400000F134EF15F00401320E826F5CEC0FF0F0
:102A500045EC38F004012C0E826F5CEC0FF0FF0E99
:102A6000D4EC0BF0E8CF00F1E8EC37F031C182F4A0
:102A70000401300E82275CEC0FF032C182F40401B5
:102A8000300E82275CEC0FF033C182F40401300E6B
:102A900082275CEC0FF07AEF30F003018351300AAB
:102AA000D8B4F2EF16F003018351310AD8B429EFFC
:102AB00017F003018351320AD8B4DEEF18F0030196
:102AC0008351330AD8B493EF1AF003018351340AC7
:102AD000D8B439EF1BF003018351730AD8B4D4EF93
:102AE00015F003018351760AD8B4D6EF15F003012F
:102AF0008351740AD8B4C1EF15F003018351540A0D
:102B0000D8B486EF15F0D8A47CEF30F00401760E2F
:102B1000826F5CEC0FF00401540E826F5CEC0FF0DE
:102B200007840001880E0C6E86EC38F029810301C1
:102B300084512D0AD8B49FEF15F00101299185C366
:102B40002FF186C330F187C331F188C332F189C3D5
:102B500033F193EC38F00AEC38F000C10BF0BDEC27
:102B60000BF001C10BF0BDEC0BF0880ED4EC0BF0B8
:102B7000E8CF40F6890ED4EC0BF0E8CF41F6CCEF6D
:102B800015F00401760E826F5CEC0FF00401740EF8
:102B9000826F5CEC0FF007840001880E0C6EDBEC9A
:102BA0000BF007948EEF26F0D4EC15F00401760EAE
:102BB000826F5CEC0FF00401760E826F5CEC0FF01C
:102BC0000784A2EC34F004012C0E826F5CEC0FF051
:102BD0000101036B026B3BC601F13AC600F101AF84
:102BE000F7EF15F00101FF0E026FFF0E036FE8EC27
:102BF00037F02967FEEF15F003EF16F004012D0EF4
:102C0000826F5CEC0FF02FC182F40401300E82273A
:102C10005CEC0FF030C182F40401300E82275CECD2
:102C20000FF031C182F40401300E82275CEC0FF00A
:102C300032C182F40401300E82275CEC0FF033C104
:102C400082F40401300E82275CEC0FF004012C0E9C
:102C5000826F5CEC0FF00101036B026B3DC601F16A
:102C60003CC600F101AF3AEF16F00101FF0E026F12
:102C7000FF0E036FE8EC37F0296741EF16F046EFDF
:102C800016F004012D0E826F5CEC0FF02FC182F460
:102C90000401300E82275CEC0FF030C182F4040195
:102CA000300E82275CEC0FF031C182F40401300E4B
:102CB00082275CEC0FF032C182F40401300E8227CF
:102CC0005CEC0FF033C182F40401300E82275CEC1F
:102CD0000FF004012C0E826F5CEC0FF00101036B0E
:102CE000026B3FC601F13EC600F101AF7DEF16F069
:102CF0000101FF0E026FFF0E036FE8EC37F029674A
:102D000084EF16F089EF16F004012D0E826F5CEC53
:102D10000FF02FC182F40401300E82275CEC0FF01B
:102D200030C182F40401300E82275CEC0FF031C117
:102D300082F40401300E82275CEC0FF032C182F481
:102D40000401300E82275CEC0FF033C182F40401E1
:102D5000300E82275CEC0FF004012C0E826F5CECCD
:102D60000FF00101036B026B37C601F136C600F1AB
:102D700001AFC0EF16F00101FF0E026FFF0E036FEF
:102D8000E8EC37F02967C7EF16F0CCEF16F0040136
:102D90002D0E826F5CEC0FF02FC182F40401300E17
:102DA00082275CEC0FF030C182F40401300E8227E0
:102DB0005CEC0FF031C182F40401300E82275CEC30
:102DC0000FF032C182F40401300E82275CEC0FF068
:102DD00033C182F40401300E82275CEC0FF00794BB
:102DE0008EEF26F00401760E826F5CEC0FF004018A
:102DF000300E826F5CEC0FF004012C0E826F5CECE5
:102E00000FF0B3EC38F045EC38F000C600F101C625
:102E100001F1E8EC37F030C182F40401300E822772
:102E20005CEC0FF031C182F40401300E82275CECBF
:102E30000FF032C182F40401300E82275CEC0FF0F7
:102E400033C182F40401300E82275CEC0FF08EEF68
:102E500026F00401760E826F5CEC0FF00401310E57
:102E6000826F5CEC0FF007840101036B026B02C6FA
:102E700000F103C601F101AF42EF17F0FF0E026F40
:102E8000FF0E036F0101076B066B04C604F105C654
:102E900005F105AF50EF17F0FF0E066FFF0E076F3D
:102EA0004FEC37F00101076B066B06C604F107C64D
:102EB00005F105AF60EF17F0FF0E066FFF0E076F0D
:102EC0004FEC37F00101076B066B08C604F109C629
:102ED00005F105AF70EF17F0FF0E066FFF0E076FDD
:102EE0004FEC37F0D8900101033302330133003344
:102EF000D8900101033302330133003304012C0E57
:102F0000826F5CEC0FF00101036B026B01C101F1F8
:102F100000C100F101AF92EF17F00101FF0E026F47
:102F2000FF0E036FE8EC37F0296799EF17F09EEF7B
:102F300017F004012D0E826F5CEC0FF02FC182F4AC
:102F40000401300E82275CEC0FF030C182F40401E2
:102F5000300E82275CEC0FF031C182F40401300E98
:102F600082275CEC0FF032C182F40401300E82271C
:102F70005CEC0FF033C182F40401300E82275CEC6C
:102F80000FF00101036B026B0AC600F10BC601F1E1
:102F900001AFCFEF17F0FF0E026FFF0E036F0101BD
:102FA000076B066B0CC604F10DC605F105AFDDEF2E
:102FB00017F0FF0E066FFF0E076F4FEC37F00101A1
:102FC000076B066B0EC604F10FC605F105AFEDEFFA
:102FD00017F0FF0E066FFF0E076F4FEC37F0010181
:102FE000076B066B10C604F111C605F105AFFDEFC6
:102FF00017F0FF0E066FFF0E076F4FEC37F0D890FB
:1030000001010333023301330033D890010103334C
:1030100002330133003304012C0E826F5CEC0FF09D
:103020000101036B026B01C101F100C100F101AFAD
:103030001FEF18F00101FF0E026FFF0E036FE8ECA7
:1030400037F0296726EF18F02BEF18F004012D0E4A
:10305000826F5CEC0FF02FC182F40401300E8227E6
:103060005CEC0FF030C182F40401300E82275CEC7E
:103070000FF031C182F40401300E82275CEC0FF0B6
:1030800032C182F40401300E82275CEC0FF033C1B0
:1030900082F40401300E82275CEC0FF00101036B17
:1030A000026B12C600F113C601F101AF5CEF18F01C
:1030B000FF0E026FFF0E036F0101076B066B14C654
:1030C00004F115C605F105AF6AEF18F0FF0E066FA3
:1030D000FF0E076F4FEC37F00101076B066B16C64A
:1030E00004F117C605F105AF7AEF18F0FF0E066F71
:1030F000FF0E076F4FEC37F00101076B066B18C628
:1031000004F119C605F105AF8AEF18F0FF0E066F3E
:10311000FF0E076F4FEC37F0D890010103330233F5
:1031200001330033D89001010333023301330033FC
:1031300004012C0E826F5CEC0FF00101036B026B3B
:1031400001C101F100C100F101AFACEF18F00101C4
:10315000FF0E026FFF0E036FE8EC37F02967B3EF45
:1031600018F0B8EF18F004012D0E826F5CEC0FF030
:103170002FC182F40401300E82275CEC0FF030C1C5
:1031800082F40401300E82275CEC0FF031C182F42E
:103190000401300E82275CEC0FF032C182F404018E
:1031A000300E82275CEC0FF033C182F40401300E44
:1031B00082275CEC0FF007948EEF26F00401760E68
:1031C000826F5CEC0FF00401320E826F5CEC0FF04A
:1031D00007840101036B026B1AC600F11BC601F1E3
:1031E00001AFF7EF18F0FF0E026FFF0E036F010142
:1031F000076B066B1CC604F11DC605F105AF05EF94
:1032000019F0FF0E066FFF0E076F4FEC37F001014C
:10321000076B066B1EC604F11FC605F105AF15EF5F
:1032200019F0FF0E066FFF0E076F4FEC37F001012C
:10323000076B066B20C604F121C605F105AF25EF2B
:1032400019F0FF0E066FFF0E076F4FEC37F0D890A6
:1032500001010333023301330033D89001010333FA
:1032600002330133003304012C0E826F5CEC0FF04B
:103270000101036B026B01C101F100C100F101AF5B
:1032800047EF19F00101FF0E026FFF0E036FE8EC2C
:1032900037F029674EEF19F053EF19F004012D0EA6
:1032A000826F5CEC0FF02FC182F40401300E822794
:1032B0005CEC0FF030C182F40401300E82275CEC2C
:1032C0000FF031C182F40401300E82275CEC0FF064
:1032D00032C182F40401300E82275CEC0FF033C15E
:1032E00082F40401300E82275CEC0FF00101036BC5
:1032F000026B22C600F123C601F101AF84EF19F081
:10330000FF0E026FFF0E036F0101076B066B24C6F1
:1033100004F125C605F105AF92EF19F0FF0E066F17
:10332000FF0E076F4FEC37F00101076B066B26C6E7
:1033300004F127C605F105AFA2EF19F0FF0E066FE5
:10334000FF0E076F4FEC37F00101076B066B28C6C5
:1033500004F129C605F105AFB2EF19F0FF0E066FB3
:10336000FF0E076F4FEC37F0D890010103330233A3
:1033700001330033D89001010333023301330033AA
:1033800004012C0E826F5CEC0FF00101036B026BE9
:1033900001C101F100C100F101AFD4EF19F0010149
:1033A000FF0E026FFF0E036FE8EC37F02967DBEFCB
:1033B00019F0E0EF19F004012D0E826F5CEC0FF0B4
:1033C0002FC182F40401300E82275CEC0FF030C173
:1033D00082F40401300E82275CEC0FF031C182F4DC
:1033E0000401300E82275CEC0FF032C182F404013C
:1033F000300E82275CEC0FF033C182F40401300EF2
:1034000082275CEC0FF00101036B026B2AC600F10E
:103410002BC601F101AF11EF1AF0FF0E026FFF0E84
:10342000036F0101076B066B2CC604F12DC605F175
:1034300005AF1FEF1AF0FF0E066FFF0E076F4FEC80
:1034400037F00101076B066B2EC604F12FC605F19C
:1034500005AF2FEF1AF0FF0E066FFF0E076F4FEC50
:1034600037F00101076B066B30C604F131C605F178
:1034700005AF3FEF1AF0FF0E066FFF0E076F4FEC20
:1034800037F0D89001010333023301330033D89071
:103490000101033302330133003304012C0E826F28
:1034A0005CEC0FF00101036B026B01C101F100C183
:1034B00000F101AF61EF1AF00101FF0E026FFF0E84
:1034C000036FE8EC37F0296768EF1AF06DEF1AF038
:1034D00004012D0E826F5CEC0FF02FC182F4040109
:1034E000300E82275CEC0FF030C182F40401300E04
:1034F00082275CEC0FF031C182F40401300E822788
:103500005CEC0FF032C182F40401300E82275CECD7
:103510000FF033C182F40401300E82275CEC0FF00F
:1035200007948EEF26F00401760E826F5CEC0FF0AC
:103530000401330E826F5CEC0FF004012C0E826FDD
:103540005CEC0FF085C382F45CEC0FF0640E0D6E42
:1035500003018551320A02E16A0E0D6E03018551A5
:10356000330A02E1700E0D6E03018551340A02E147
:10357000760E0D6E03018551350A02E17C0E0D6E4B
:1035800003018551360A02E1820E0D6E0301865158
:10359000780A65E00DC00CF086EC38F02981030153
:1035A00087512D0AD8B4D7EF1AF00101299188C3A9
:1035B0002FF189C330F18AC331F18BC332F18CC34F
:1035C00033F193EC38F00AEC38F000C10BF0BDECAD
:1035D0000BF001C10BF0BDEC0BF086EC38F029814B
:1035E00003018E512D0AD8B4F8EF1AF00101299188
:1035F0008FC32FF190C330F191C331F192C332F1F7
:1036000093C333F193EC38F00AEC38F000C10BF0BF
:10361000BDEC0BF001C10BF0BDEC0BF086EC38F00B
:103620002981030195512D0AD8B419EF1BF001012E
:10363000299196C32FF197C330F198C331F199C303
:1036400032F19AC333F193EC38F00AEC38F000C150
:103650000BF0BDEC0BF001C10BF0BDEC0BF00DC09D
:103660000CF0DBEC0BF0DBEC0BF0DBEC0BF08EEF9B
:1036700026F00401760E826F5CEC0FF00401340E2C
:10368000826F5CEC0FF003018451780AD8B411EF1B
:103690001CF03E0E0C6E86EC38F02981030185513A
:1036A0002D0AD8B456EF1BF00101299186C32FF1E2
:1036B00087C330F188C331F189C332F18AC333F152
:1036C00093EC38F00AEC38F000C10BF0BDEC0BF0D5
:1036D00001C10BF0BDEC0BF086EC38F02981030141
:1036E0008C512D0AD8B477EF1BF0010129918DC3BD
:1036F0002FF18EC330F18FC331F190C332F191C3FA
:1037000033F193EC38F00AEC38F000C10BF0BDEC6B
:103710000BF001C10BF0BDEC0BF086EC38F0298109
:10372000030193512D0AD8B498EF1BF001012991A0
:1037300094C32FF195C330F196C331F197C332F1A1
:1037400098C333F193EC38F00AEC38F000C10BF079
:10375000BDEC0BF001C10BF0BDEC0BF086EC38F0CA
:10376000298103019A512D0AD8B4B9EF1BF0010148
:1037700029919BC32FF19CC330F19DC331F19EC3AE
:1037800032F19FC333F193EC38F00AEC38F000C10A
:103790000BF0BDEC0BF001C10BF0BDEC0BF086ECB7
:1037A00038F029810301A1512D0AD8B4DAEF1BF0BA
:1037B00001012991A2C32FF1A3C330F1A4C331F1B8
:1037C000A5C332F1A6C333F193EC38F00AEC38F01C
:1037D00000C10BF0BDEC0BF001C10BF0BDEC0BF028
:1037E00086EC38F029810301A8512D0AD8B4FBEFEB
:1037F0001BF001012991A9C32FF1AAC330F1ABC37A
:1038000031F1ACC332F1ADC333F193EC38F00AECD3
:1038100038F000C10BF0BDEC0BF001C10BF0BDECBA
:103820000BF03E0E0C6EDBEC0BF0DBEC0BF0DBEC8C
:103830000BF0DBEC0BF0DBEC0BF0DBEC0BF08EEFCA
:1038400026F003018351300AD8B41CEF21F00301A4
:103850008351310AD8B449EF22F003018351320A6F
:10386000D8B4B7EF22F003018351330AD8B4C7EFBD
:1038700022F003018351340AD8B4D7EF22F00301B8
:103880008351350AD8B432EF26F003018351360A4A
:10389000D8B460EF26F003018351370AD8B4F4EFAF
:1038A0001EF003018351380AD8B492EF1FF00301D0
:1038B0008351460AD8B485EF25F0030183514D0AA0
:1038C000D8B46DEF1DF0030183516D0AD8B487EFB2
:1038D0001DF0030183515A0AD8B4C3EF21F003014C
:1038E0008351490AD8B460EF27F003018351500A8D
:1038F000D8B492EF26F003018351540AD8B40BEFE9
:1039000027F003018351630AD8B4A7EF1DF0030128
:103910008351430AD8B49FEF1EF003018351730A09
:10392000D8B4A5EF1DF003018351610AD8B4BAEFF2
:103930001CF003018351650AD8B46CEF21F0030138
:103940008351450AD8B47AEF21F003018351620A0A
:10395000D8B488EF21F003018351420AD8B496EF1E
:1039600021F003018351760AD8B4A4EF21F0D8A442
:103970007CEF30F004014C0E826F5CEC0FF0040120
:10398000610E826F5CEC0FF094EC3AF004012C0EA7
:10399000826F5CEC0FF045EC38F0AFC500F101012F
:1039A000E8EC37F031C182F40401300E82275CEC80
:1039B0000FF032C182F40401300E82275CEC0FF06C
:1039C00033C182F40401300E82275CEC0FF0040155
:1039D0002C0E826F5CEC0FF045EC38F0B0C500F1B6
:1039E0000101E8EC37F031C182F40401300E822786
:1039F0005CEC0FF032C182F40401300E82275CECE3
:103A00000FF033C182F40401300E82275CEC0FF01A
:103A100004012C0E826F5CEC0FF045EC38F0B1C560
:103A200000F10101E8EC37F031C182F40401300EFD
:103A300082275CEC0FF032C182F40401300E822741
:103A40005CEC0FF033C182F40401300E82275CEC91
:103A50000FF004012C0E826F5CEC0FF045EC38F097
:103A6000B2C500F10101E8EC37F031C182F4040184
:103A7000300E82275CEC0FF032C182F40401300E6C
:103A800082275CEC0FF033C182F40401300E8227F0
:103A90005CEC0FF004012C0E826F5CEC0FF045EC37
:103AA00038F0B6C500F10101E8EC37F031C182F41D
:103AB0000401300E82275CEC0FF032C182F4040165
:103AC000300E82275CEC0FF033C182F40401300E1B
:103AD00082275CEC0FF08EEF26F086EC38F084C382
:103AE00033F193EC38F00AEC38F0200E0C6E00C184
:103AF0000BF0BDEC0BF000C12FF505012F51000AB2
:103B000006E005012F51010A02E02EEC3BF0040112
:103B10004C0E826F5CEC0FF004014D0E826F5CEC7A
:103B20000FF004012C0E826F5CEC0FF045EC38F0C6
:103B30002FC500F1E8EC37F033C182F40401300EF8
:103B400082275CEC0FF08EEF26F020EF42F00401AC
:103B50004C0E826F5CEC0FF00401630E826F5CEC24
:103B60000FF0ECEC39F004012C0E826F5CEC0FF0DE
:103B7000BCEC1DF08EEF26F045EC38F0B5C500F139
:103B80000101003B0F0E0017E8EC37F033C182F45F
:103B90000401300E82275CEC0FF0B5C500F1010185
:103BA0000F0E01010017E8EC37F033C182F4040175
:103BB000300E82275CEC0FF004012D0E826F5CEC5E
:103BC0000FF0B4C500F10101003B0F0E0017E8EC47
:103BD00037F033C182F40401300E82275CEC0FF021
:103BE000B4C500F101010F0E01010017E8EC37F038
:103BF00033C182F40401300E82275CEC0FF0040123
:103C00002D0E826F5CEC0FF0B3C500F10101003B9B
:103C10000F0E0017E8EC37F033C182F40401300EC8
:103C200082275CEC0FF0B3C500F101010F0E01011A
:103C30000017E8EC37F033C182F40401300E82271C
:103C40005CEC0FF00401200E826F5CEC0FF0B2C54B
:103C500000F10F0E01010017E8EC37F033C182F4D8
:103C60000401300E82275CEC0FF00401200E826FFD
:103C70005CEC0FF0B1C500F101010101003B0F0E3A
:103C80000017E8EC37F033C182F40401300E8227CC
:103C90005CEC0FF0B1C500F101010F0E010100173E
:103CA000E8EC37F033C182F40401300E82275CEC7B
:103CB0000FF004013A0E826F5CEC0FF0B0C500F11A
:103CC0000101003B0F0E0017E8EC37F033C182F41E
:103CD0000401300E82275CEC0FF0B0C500F1010149
:103CE0000F0E01010017E8EC37F033C182F4040134
:103CF000300E82275CEC0FF004013A0E826F5CEC10
:103D00000FF0AFC500F10101003B0F0E0017E8EC0A
:103D100037F033C182F40401300E82275CEC0FF0DF
:103D2000AFC500F101010F0E0017E8EC37F033C109
:103D300082F40401300E82275CEC0FF0120084C381
:103D4000E8FF0F0BE83AE8CFB5F585C3E8FF0F0BA6
:103D50000501B51387C3E8FF0F0BE83AE8CFB4F5C8
:103D600088C3E8FF0F0B0501B4138AC3E8FF0F0BEC
:103D7000E83AE8CFB3F58BC3E8FF0F0B0501B313A7
:103D80008DC3E8FF0F0BE8CFB2F58FC3E8FF0F0B31
:103D9000E83AE8CFB1F590C3E8FF0F0B0501B11386
:103DA00092C3E8FF0F0BE83AE8CFB0F593C3E8FF02
:103DB0000F0B0501B01395C3E8FF0F0BE83AE8CFEE
:103DC000AFF596C3E8FF0F0B0501AF1347EC3AF0D0
:103DD00004014C0E826F5CEC0FF00401430E826F05
:103DE0005CEC0FF0B1EF1DF0078404014C0E826F04
:103DF0005CEC0FF00401370E826F5CEC0FF00401F5
:103E00002C0E826F5CEC0FF005012E51130A06E0B8
:103E100005012E51170A0DE08FEF1FF00101000E72
:103E2000006F000E016F100E026F000E036F22EF85
:103E30001FF00101000E006F000E016F000E026FF7
:103E4000010E036FE8EC37F02AC182F40401300E52
:103E500082275CEC0FF02BC182F40401300E822724
:103E60005CEC0FF02CC182F40401300E82275CEC74
:103E70000FF02DC182F40401300E82275CEC0FF0AC
:103E80002EC182F40401300E82275CEC0FF02FC1AA
:103E900082F40401300E82275CEC0FF030C182F412
:103EA0000401300E82275CEC0FF031C182F4040172
:103EB000300E82275CEC0FF032C182F40401300E28
:103EC00082275CEC0FF033C182F40401300E8227AC
:103ED0005CEC0FF004012C0E826F5CEC0FF0010122
:103EE000200E006F000E016F000E026F000E036FB8
:103EF000E8EC37F031C182F40401300E82275CEC2B
:103F00000FF032C182F40401300E82275CEC0FF016
:103F100033C182F40401300E82275CEC0FF0079469
:103F20008EEF26F00501216B226B236B246B0401BD
:103F30004C0E826F5CEC0FF00401380E826F5CEC6B
:103F40000FF004012C0E826F5CEC0FF00101200ECB
:103F5000006F000E016F000E026F000E036FE8ECA1
:103F600037F02AC182F40401300E82275CEC0FF096
:103F70002BC182F40401300E82275CEC0FF02CC1BF
:103F800082F40401300E82275CEC0FF02DC182F424
:103F90000401300E82275CEC0FF02EC182F4040184
:103FA000300E82275CEC0FF02FC182F40401300E3A
:103FB00082275CEC0FF030C182F40401300E8227BE
:103FC0005CEC0FF031C182F40401300E82275CEC0E
:103FD0000FF032C182F40401300E82275CEC0FF046
:103FE00033C182F40401300E82275CEC0FF004012F
:103FF0002C0E826F5CEC0FF025C500F126C501F197
:1040000027C502F128C503F10101200E046F000E3F
:10401000056F000E066F000E076F7BEC37F000C1D6
:1040200033F501C134F502C135F503C136F5E8ECCD
:1040300037F02AC182F40401300E82275CEC0FF0C5
:104040002BC182F40401300E82275CEC0FF02CC1EE
:1040500082F40401300E82275CEC0FF02DC182F453
:104060000401300E82275CEC0FF02EC182F40401B3
:10407000300E82275CEC0FF02FC182F40401300E69
:1040800082275CEC0FF030C182F40401300E8227ED
:104090005CEC0FF031C182F40401300E82275CEC3D
:1040A0000FF032C182F40401300E82275CEC0FF075
:1040B00033C182F40401300E82275CEC0FF066EC11
:1040C0000FF0050133676CEF20F034676CEF20F0E0
:1040D00035676CEF20F0366702D00BEF21F0129EAF
:1040E000129C21C500F122C501F123C502F124C5AE
:1040F00003F1899A400EC76E200EC66E9E96C69E2C
:104100000B0EC96EFF0E9EB602D0E82EFCD79E960F
:10411000C69E02C1C9FFFF0E9EB602D0E82EFCD794
:104120009E96C69E01C1C9FFFF0E9EB602D0E82E24
:10413000FCD79E96C69E00C1C9FFFF0E9EB602D058
:10414000E82EFCD79E96C69EC952FF0E9EB602D0A0
:10415000E82EFCD70501200E326F040114EE00F0AA
:1041600080517F0BE1269E96C69EC952FF0E9EB6D9
:1041700002D0E82EFCD7C9CFE7FF0401802B050150
:10418000322FADEF20F0898A33C500F134C501F13B
:1041900035C502F136C503F10101010E046F000EB1
:1041A000056F000E066F000E076F4AEC37F000C176
:1041B00033F501C134F502C135F503C136F505010A
:1041C0003367EAEF20F03467EAEF20F03567EAEF73
:1041D00020F0366702D00BEF21F021C500F122C597
:1041E00001F123C502F124C503F10101200E046F82
:1041F000000E056F000E066F000E076F4FEC37F0D4
:1042000000C121F501C122F502C123F503C124F546
:10421000128E7CEF30F00401450E826F5CEC0FF0E3
:1042200004014F0E826F5CEC0FF00401460E826FAA
:104230005CEC0FF08EEF26F00784E1EC41F045ECEA
:1042400038F02DC500F1E8EC37F004014C0E826F18
:104250005CEC0FF00401300E826F5CEC0FF0040197
:104260002C0E826F5CEC0FF031C182F40401300E31
:1042700082275CEC0FF032C182F40401300E8227F9
:104280005CEC0FF033C182F40401300E82275CEC49
:104290000FF004012C0E826F5CEC0FF045EC38F04F
:1042A0002EC500F1E8EC37F031C182F40401300E84
:1042B00082275CEC0FF032C182F40401300E8227B9
:1042C0005CEC0FF033C182F40401300E82275CEC09
:1042D0000FF007948EEF26F004014C0E826F5CEC19
:1042E0000FF00401650E826F5CEC0FF00AEC3CF0FD
:1042F0008EEF26F004014C0E826F5CEC0FF004018F
:10430000450E826F5CEC0FF021EC3CF08EEF26F056
:1043100004014C0E826F5CEC0FF00401620E826FA0
:104320005CEC0FF04FEC3CF08EEF26F004014C0EED
:10433000826F5CEC0FF00401420E826F5CEC0FF0B8
:1043400038EC3CF08EEF26F004014C0E826F5CECF2
:104350000FF00401760E826F5CEC0FF004012C0E5E
:10436000826F5CEC0FF010A807D00401310E826F51
:104370005CEC0FF08EEF26F00401300E826F5CECE7
:104380000FF08EEF26F004014C0E826F5CEC0FF004
:1043900004015A0E826F5CEC0FF004012C0E826F48
:1043A0005CEC0FF0E1EC41F045EC38F005012E51EA
:1043B000130A06E005012E51170A0DE0F4EF21F073
:1043C0000101000E006F000E016F100E026F000E53
:1043D000036FF4EF21F00101000E006F000E016F7A
:1043E000000E026F010E036F0101200E046F000E1C
:1043F000056F000E066F000E076F7BEC37F0E8ECE0
:1044000037F02AC182F40401300E82275CEC0FF0F1
:104410002BC182F40401300E82275CEC0FF02CC11A
:1044200082F40401300E82275CEC0FF02DC182F47F
:104430000401300E82275CEC0FF02EC182F40401DF
:10444000300E82275CEC0FF02FC182F40401300E95
:1044500082275CEC0FF030C182F40401300E822719
:104460005CEC0FF031C182F40401300E82275CEC69
:104470000FF032C182F40401300E82275CEC0FF0A1
:1044800033C182F40401300E82275CEC0FF08EEF12
:1044900026F0078404014C0E826F5CEC0FF00401DF
:1044A000310E826F5CEC0FF004012C0E826F5CEC1D
:1044B0000FF025C500F126C501F127C502F128C579
:1044C00003F10101200E046F000E056F000E066F50
:1044D000000E076F7BEC37F0E8EC37F02AC182F46E
:1044E0000401300E82275CEC0FF02BC182F4040132
:1044F000300E82275CEC0FF02CC182F40401300EE8
:1045000082275CEC0FF02DC182F40401300E82276B
:104510005CEC0FF02EC182F40401300E82275CECBB
:104520000FF02FC182F40401300E82275CEC0FF0F3
:1045300030C182F40401300E82275CEC0FF031C1EF
:1045400082F40401300E82275CEC0FF032C182F459
:104550000401300E82275CEC0FF033C182F40401B9
:10456000300E82275CEC0FF007948EEF26F0078464
:1045700004014C0E826F5CEC0FF00401320E826F6E
:104580005CEC0FF03DEC3EF007948EEF26F00784D4
:1045900004014C0E826F5CEC0FF00401330E826F4D
:1045A0005CEC0FF09AEC3EF0079454EF22F0078495
:1045B00004014C0E826F5CEC0FF00401340E826F2C
:1045C0005CEC0FF004012C0E826F5CEC0FF086ECBB
:1045D00038F084C32AF185C32BF186C32CF187C33D
:1045E0002DF188C32EF189C32FF18AC330F18BC31B
:1045F00031F18CC332F18DC333F10101296B93EC9E
:1046000038F00AEC38F0200E046F000E056F000E33
:10461000066F000E076F5BEC37F000C121F501C19A
:1046200022F502C123F503C124F594EC41F038C50D
:10463000AFF539C5B0F53AC5B1F53BC5B2F53CC5E6
:10464000B3F53DC5B4F53EC5B5F5BCEC1DF00401B0
:104650002C0E826F5CEC0FF03FC500F140C501F1FC
:1046600041C502F142C503F10101000E046F000EC5
:10467000056F010E066F000E076F7BEC37F0E8EC5C
:1046800037F0296746EF23F04BEF23F004012D0E9E
:10469000826F5CEC0FF030C182F40401300E82278F
:1046A0005CEC0FF031C182F40401300E82275CEC27
:1046B0000FF004012E0E826F5CEC0FF032C182F419
:1046C0000401300E82275CEC0FF033C182F4040148
:1046D000300E82275CEC0FF004012C0E826F5CEC34
:1046E0000FF045EC38F043C500F144C501F1A6ECEC
:1046F00031F004012C0E826F5CEC0FF045EC38F0C9
:1047000045C500F1E8EC37F031C182F40401300E08
:1047100082275CEC0FF032C182F40401300E822754
:104720005CEC0FF033C182F40401300E82275CECA4
:104730000FF004012C0E826F5CEC0FF00101036B93
:10474000026B4CC501F14BC500F101AFADEF23F099
:104750000101FF0E026FFF0E036FE8EC37F02967CF
:10476000B4EF23F0B9EF23F004012D0E826F5CEC5F
:104770000FF02FC182F40401300E82275CEC0FF0A1
:1047800030C182F40401300E82275CEC0FF031C19D
:1047900082F40401300E82275CEC0FF032C182F407
:1047A0000401300E82275CEC0FF033C182F4040167
:1047B000300E82275CEC0FF004012C0E826F5CEC53
:1047C0000FF00101036B026B4EC501F14DC500F105
:1047D00001AFF0EF23F00101FF0E026FFF0E036F38
:1047E000E8EC37F02967F7EF23F0FCEF23F0040142
:1047F0002D0E826F5CEC0FF02FC182F40401300E9D
:1048000082275CEC0FF030C182F40401300E822765
:104810005CEC0FF031C182F40401300E82275CECB5
:104820000FF032C182F40401300E82275CEC0FF0ED
:1048300033C182F40401300E82275CEC0FF00401D6
:104840002C0E826F5CEC0FF00101036B026B50C504
:1048500001F14FC500F101AF33EF24F00101FF0E6C
:10486000026FFF0E036FE8EC37F029673AEF24F090
:104870003FEF24F004012D0E826F5CEC0FF02FC18E
:1048800082F40401300E82275CEC0FF030C182F418
:104890000401300E82275CEC0FF031C182F4040178
:1048A000300E82275CEC0FF032C182F40401300E2E
:1048B00082275CEC0FF033C182F40401300E8227B2
:1048C0005CEC0FF004012C0E826F5CEC0FF0010128
:1048D000036B026B52C501F151C500F101AF76EFD8
:1048E00024F00101FF0E026FFF0E036FE8EC37F0BA
:1048F00029677DEF24F082EF24F004012D0E826FF2
:104900005CEC0FF02FC182F40401300E82275CECC6
:104910000FF030C182F40401300E82275CEC0FF0FE
:1049200031C182F40401300E82275CEC0FF032C1F9
:1049300082F40401300E82275CEC0FF033C182F464
:104940000401300E82275CEC0FF004012C0E826F04
:104950005CEC0FF00101036B026B54C501F153C510
:1049600000F101AFB9EF24F00101FF0E026FFF0E5D
:10497000036FE8EC37F02967C0EF24F0C5EF24F0AF
:1049800004012D0E826F5CEC0FF02FC182F4040144
:10499000300E82275CEC0FF030C182F40401300E3F
:1049A00082275CEC0FF031C182F40401300E8227C3
:1049B0005CEC0FF032C182F40401300E82275CEC13
:1049C0000FF033C182F40401300E82275CEC0FF04B
:1049D00004012C0E826F5CEC0FF00101036B026B83
:1049E00056C501F155C500F101AFFCEF24F00101FE
:1049F000FF0E026FFF0E036FE8EC37F0296703EF3D
:104A000025F008EF25F004012D0E826F5CEC0FF00D
:104A10002FC182F40401300E82275CEC0FF030C10C
:104A200082F40401300E82275CEC0FF031C182F475
:104A30000401300E82275CEC0FF032C182F40401D5
:104A4000300E82275CEC0FF033C182F40401300E8B
:104A500082275CEC0FF004012C0E826F5CEC0FF0EF
:104A60000101036B026B4AC501F149C500F101AFB9
:104A70003FEF25F00101FF0E026FFF0E036FE8EC20
:104A800037F0296746EF25F04BEF25F004012D0E96
:104A9000826F5CEC0FF02FC182F40401300E82278C
:104AA0005CEC0FF030C182F40401300E82275CEC24
:104AB0000FF031C182F40401300E82275CEC0FF05C
:104AC00032C182F40401300E82275CEC0FF033C156
:104AD00082F40401300E82275CEC0FF004012C0EEE
:104AE000826F5CEC0FF037C5E8FFE8B806D0040130
:104AF000300E826F5CEC0FF005D00401310E826F36
:104B00005CEC0FF007948EEF26F086EC38F085C34E
:104B10002AF186C32BF187C32CF188C32DF189C3F9
:104B20002EF18AC32FF18BC330F18CC331F18DC3C9
:104B300032F18EC333F10101296B93EC38F00AECAA
:104B400038F00101010E046F000E056F000E066FB4
:104B5000000E076F4AEC37F0100E046F000E056F61
:104B6000000E066F000E076F5BEC37F000C129F5F1
:104B700001C12AF502C12BF503C12CF5C4EC3DF0AF
:104B800004014C0E826F5CEC0FF00401460E826F44
:104B90005CEC0FF004012C0E826F5CEC0FF025C56D
:104BA00000F126C501F127C502F128C503F1010175
:104BB000100E046F000E056F000E066F000E076FDB
:104BC0007BEC37F0E8EC37F02AC182F40401300EB8
:104BD00082275CEC0FF02BC182F40401300E822797
:104BE0005CEC0FF02CC182F40401300E82275CECE7
:104BF0000FF02DC182F40401300E82275CEC0FF01F
:104C00002EC182F40401300E82275CEC0FF02FC11C
:104C100082F40401300E82275CEC0FF030C182F484
:104C20000401300E82275CEC0FF031C182F40401E4
:104C3000300E82275CEC0FF032C182F40401300E9A
:104C400082275CEC0FF033C182F40401300E82271E
:104C50005CEC0FF08EEF26F00F989AEC3EF030806F
:104C60007CEF30F004014C0E826F5CEC0FF004011D
:104C7000350E826F5CEC0FF004012C0E826F5CEC41
:104C80000FF045EC38F00784B9C500F10794E8EC63
:104C900037F031C182F40401300E82275CEC0FF052
:104CA00032C182F40401300E82275CEC0FF033C174
:104CB00082F40401300E82275CEC0FF08EEF26F0B8
:104CC0005DEC3EF045EC38F037C500F1E8EC37F02C
:104CD00004014C0E826F5CEC0FF00401360E826F03
:104CE0005CEC0FF004012C0E826F5CEC0FF031C114
:104CF00082F40401300E82275CEC0FF032C182F4A2
:104D00000401300E82275CEC0FF033C182F4040101
:104D1000300E82275CEC0FF08EEF26F066EC0FF081
:104D20007CEF30F004014C0E826F5CEC0FF004015C
:104D3000500E826F5CEC0FF004012C0E826F5CEC65
:104D40000FF085C32AF186C32BF187C32CF188C3EA
:104D50002DF189C32EF18AC32FF18BC330F18CC39F
:104D600031F18DC332F18EC333F1010193EC38F090
:104D70000AEC38F003018451530A0DE00301845119
:104D80004D0A38E00401780E826F5CEC0FF066EC9F
:104D90000FF07CEF30F00401530E826F5CEC0FF0EB
:104DA000250E0C6E00C10BF0BDEC0BF0260E0C6E48
:104DB00001C10BF0BDEC0BF0270E0C6E02C10BF025
:104DC000BDEC0BF0280E0C6E03C10BF0BDEC0BF02C
:104DD00000C157F501C158F502C159F503C15AF593
:104DE00000C15BF501C15CF502C15DF503C15EF573
:104DF0006FEF27F004014D0E826F5CEC0FF0290E6F
:104E00000C6E00C10BF0BDEC0BF000C15FF500C1F2
:104E100060F56FEF27F004014C0E826F5CEC0FF031
:104E20000401540E826F5CEC0FF004012C0E826FB3
:104E30005CEC0FF084C32AF185C32BF186C32CF1FF
:104E400087C32DF188C32EF189C32FF18AC330F1B6
:104E50008BC331F18DC332F18EC333F1010193EC79
:104E600038F00AEC38F00101000E046F000E056FF7
:104E7000010E066F000E076F5BEC37F0210E0C6E13
:104E800000C10BF0BDEC0BF0220E0C6E01C10BF05B
:104E9000BDEC0BF0230E0C6E02C10BF0BDEC0BF061
:104EA000240E0C6E03C10BF0BDEC0BF000C161F5DC
:104EB00001C162F502C163F503C164F56FEF27F02C
:104EC00004014C0E826F5CEC0FF00401490E826FFE
:104ED0005CEC0FF004012C0E826F5CEC0FF0250EE1
:104EE000D4EC0BF0E8CF00F1260ED4EC0BF0E8CFB9
:104EF00001F1270ED4EC0BF0E8CF02F1280ED4EC30
:104F00000BF0E8CF03F1E8EC37F0ABEC35F004013F
:104F1000730E826F5CEC0FF004012C0E826F5CEC60
:104F20000FF045EC38F0290ED4EC0BF0E8CF00F18F
:104F3000E8EC37F0ABEC35F004016D0E826F5CEC01
:104F40000FF004012C0E826F5CEC0FF05BC500F1DA
:104F50005CC501F15DC502F15EC503F1E8EC37F017
:104F6000ABEC35F00401730E826F5CEC0FF00401C2
:104F70002C0E826F5CEC0FF045EC38F060C500F150
:104F8000E8EC37F0ABEC35F004016D0E826F5CECB1
:104F90000FF004012C0E826F5CEC0FF061C500F184
:104FA00062C501F163C502F164C503F197EC30F00D
:104FB00004012C0E826F5CEC0FF066EC0FF07CEFBE
:104FC00030F083C32AF184C32BF185C32CF186C34F
:104FD0002DF187C32EF188C32FF189C330F18AC325
:104FE00031F18BC332F18CC333F1010193EC38F012
:104FF0000AEC38F0160E0C6E00C10BF0BDEC0BF095
:10500000170E0C6E01C10BF0BDEC0BF0180E0C6E00
:1050100002C10BF0BDEC0BF0190E0C6E03C10BF0CE
:10502000BDEC0BF000C18EF101C18FF102C190F116
:1050300003C191F100C192F101C193F102C194F158
:1050400003C195F1C3EF28F083C32AF184C32BF188
:1050500085C32CF186C32DF187C32EF188C32FF1B0
:1050600089C330F18AC331F18BC332F18CC333F180
:10507000010193EC38F00AEC38F000C18EF101C167
:105080008FF102C190F103C191F100C192F101C110
:1050900093F102C194F103C195F1C3EF28F083C3EA
:1050A0002AF184C32BF185C32CF186C32DF187C36C
:1050B0002EF188C32FF189C330F18AC331F18CC33B
:1050C00032F18DC333F1010193EC38F00AEC38F082
:1050D0000101000E046F000E056F010E066F000E39
:1050E000076F5BEC37F01A0E0C6E00C10BF0BDECD5
:1050F0000BF01B0E0C6E01C10BF0BDEC0BF01C0E87
:105100000C6E02C10BF0BDEC0BF01D0E0C6E03C15A
:105110000BF0BDEC0BF000C196F101C197F102C19B
:1051200098F103C199F1C3EF28F083C32AF184C336
:105130002BF185C32CF186C32DF187C32EF188C3D3
:105140002FF189C330F18AC331F18CC332F18DC3A1
:1051500033F1010193EC38F00AEC38F00101000E54
:10516000046F000E056F010E066F000E076F5BECFB
:1051700037F000C196F101C197F102C198F103C166
:1051800099F1C3EF28F0160ED4EC0BF0E8CF00F144
:10519000170ED4EC0BF0E8CF01F1180ED4EC0BF0A5
:1051A000E8CF02F1190ED4EC0BF0E8CF03F1E8ECF4
:1051B00037F0ABEC35F00401730E826F5CEC0FF04E
:1051C00004012C0E826F5CEC0FF08EC100F18FC1D8
:1051D00001F190C102F191C103F1E8EC37F0ABECC1
:1051E00035F00401730E826F5CEC0FF004012C0E9D
:1051F000826F5CEC0FF01A0ED4EC0BF0E8CF00F1EC
:105200001B0ED4EC0BF0E8CF01F11C0ED4EC0BF02C
:10521000E8CF02F11D0ED4EC0BF0E8CF03F197ECD0
:1052200030F004012C0E826F5CEC0FF096C100F19F
:1052300097C101F198C102F199C103F197EC30F0E7
:1052400066EC0FF07CEF30F00401690E826F5CECCD
:105250000FF004012C0E826F5CEC0FF00101040EC4
:10526000006F000E016F000E026F000E036FE8EC7E
:1052700037F02CC182F40401300E82275CEC0FF071
:105280002DC182F40401300E82275CEC0FF02EC198
:1052900082F40401300E82275CEC0FF02FC182F4FF
:1052A0000401300E82275CEC0FF030C182F404015F
:1052B000300E82275CEC0FF031C182F40401300E15
:1052C00082275CEC0FF032C182F40401300E822799
:1052D0005CEC0FF033C182F40401300E82275CECE9
:1052E0000FF004012C0E826F5CEC0FF001010B0E2D
:1052F000006F000E016F000E026F000E036FE8ECEE
:1053000037F02CC182F40401300E82275CEC0FF0E0
:105310002DC182F40401300E82275CEC0FF02EC107
:1053200082F40401300E82275CEC0FF02FC182F46E
:105330000401300E82275CEC0FF030C182F40401CE
:10534000300E82275CEC0FF031C182F40401300E84
:1053500082275CEC0FF032C182F40401300E822708
:105360005CEC0FF033C182F40401300E82275CEC58
:105370000FF004012C0E826F5CEC0FF001013A0E6D
:10538000006F000E016F000E026F000E036FE8EC5D
:1053900037F02CC182F40401300E82275CEC0FF050
:1053A0002DC182F40401300E82275CEC0FF02EC177
:1053B00082F40401300E82275CEC0FF02FC182F4DE
:1053C0000401300E82275CEC0FF030C182F404013E
:1053D000300E82275CEC0FF031C182F40401300EF4
:1053E00082275CEC0FF032C182F40401300E822778
:1053F0005CEC0FF033C182F40401300E82275CECC8
:105400000FF004012C0E826F5CEC0FF0200EF86E92
:10541000F76AF66A04010900F5CF82F45CEC0FF03C
:105420000900F5CF82F45CEC0FF00900F5CF82F4AF
:105430005CEC0FF00900F5CF82F45CEC0FF0090092
:10544000F5CF82F45CEC0FF00900F5CF82F45CEC50
:105450000FF00900F5CF82F45CEC0FF00900F5CFF6
:1054600082F45CEC0FF066EC0FF07CEF30F08351CF
:10547000630AD8A47AEF30F08451610AD8A47AEF95
:1054800030F085516C0AD8A47AEF30F08651410A89
:105490003FE08651440A1BE08651420AD8B49BEF94
:1054A0002AF08651350AD8B406EF32F08651360A12
:1054B000D8B45BEF32F08651370AD8B4C4EF32F07B
:1054C0008651380AD8B422EF33F07AEF30F00798DB
:1054D000079A04017A0E826F5CEC0FF00401780EDB
:1054E000826F5CEC0FF00401640E826F5CEC0FF0D5
:1054F0000401550E826F5CEC0FF084EF2AF004017A
:105500004C0E826F5CEC0FF066EC0FF07CEF30F02D
:105510000788079A04017A0E826F5CEC0FF0040191
:10552000410E826F5CEC0FF00401610E826F5CEC47
:105530000FF078EF2AF00798078A04017A0E826F3D
:105540005CEC0FF00401420E826F5CEC0FF0040182
:10555000610E826F5CEC0FF078EF2AF00101666754
:10556000B9EF2AF06767B9EF2AF06867B9EF2AF058
:10557000696715D04F67C4EF2AF05067C4EF2AF06F
:105580005167C4EF2AF052670AD00101000E006F84
:10559000000E016F000E026F000E036F120011B8B3
:1055A0000AD00101620E046F010E056F000E066F36
:1055B000000E076F09D00101A70E046F020E056FE0
:1055C000000E066F000E076F66C100F167C101F1A2
:1055D00068C102F169C103F14AEC37F003BF61EF22
:1055E0002BF0119A119C0101000E046FA80E056F9B
:1055F000550E066F020E076F66C100F167C101F11B
:1056000068C102F169C103F166C18AF167C18BF11A
:1056100068C18CF169C18DF14AEC37F003BF0BD042
:105620000101000E8A6FA80E8B6F550E8C6F020E53
:105630008D6F118A119C0E0ED4EC0BF0E8CF18F18F
:105640000F0ED4EC0BF0E8CF19F1100ED4EC0BF0E8
:10565000E8CF1AF1110ED4EC0BF0E8CF1BF193EC6C
:1056600036F08AC104F18BC105F18CC106F18DC100
:1056700007F14AEC37F0078257EC36F093EC36F03E
:10568000079257EC36F08AC100F18BC101F18CC151
:1056900002F18DC103F1079257EC36F0CC0E046F86
:1056A000E00E056F870E066F050E076F4AEC37F0A8
:1056B00000C118F101C119F102C11AF103C11BF1B6
:1056C00040D013AA66EF2BF0138E139A119C119AF7
:1056D0000101800E006F1A0E016F060E026F000EA0
:1056E000036F4FC104F150C105F151C106F152C120
:1056F00007F14AEC37F003AF05D045EC38F0118CD8
:10570000119A12000E0ED4EC0BF0E8CF18F10F0E28
:10571000D4EC0BF0E8CF19F1100ED4EC0BF0E8CF7D
:105720001AF1110ED4EC0BF0E8CF1BF14FC100F1D0
:1057300050C101F151C102F152C103F1078257EC8E
:1057400036F018C100F119C101F11AC102F11BC1F3
:1057500003F112000401730E826F5CEC0FF0040180
:105760002C0E826F5CEC0FF0078462C166F163C19E
:1057700067F164C168F165C169F14BC14FF14CC17A
:1057800050F14DC151F14EC152F157C159F158C1BB
:105790005AF10794D0EC2BF066EC0FF07CEF30F070
:1057A00066C100F167C101F168C102F169C103F18D
:1057B0000101E8EC37F0ABEC35F00401630E826FC9
:1057C0005CEC0FF004012C0E826F5CEC0FF04FC10B
:1057D00000F150C101F151C102F152C103F10101C7
:1057E000E8EC37F0ABEC35F00401660E826F5CEC50
:1057F0000FF004012C0E826F5CEC0FF045EC38F0DA
:1058000059C100F15AC101F10101E8EC37F0ABECEC
:1058100035F00401740E826F5CEC0FF01200108200
:105820000401530E826F5CEC0FF004012C0E826FAA
:105830005CEC0FF083C32AF184C32BF185C32CF1F8
:1058400086C32DF187C32EF188C32FF189C330F1B0
:105850008AC331F18BC332F18CC333F1010193EC74
:1058600038F00AEC38F000C166F101C167F102C1FD
:1058700068F103C169F18EC32AF18FC32BF190C384
:105880002CF191C32DF192C32EF193C32FF194C348
:1058900030F195C331F196C332F197C333F1010171
:1058A00093EC38F00AEC38F000C14FF101C150F12F
:1058B00002C151F103C152F186EC38F099C32FF1C6
:1058C0009AC330F19BC331F19CC332F19DC333F1D4
:1058D000010193EC38F00AEC38F000C159F101C134
:1058E0005AF1D0EC2BF004012C0E826F5CEC0FF01F
:1058F0008AEF2CF0118E19A002D019AE108C18BEB0
:1059000002D018A4108E03018251520A02E10F82C4
:1059100001D00F928251750A02E1108401D01094D7
:105920008251550A02E1108601D010968351310A46
:1059300003E11382138402D01392139411A003D0B5
:1059400011A401D01084078410B208EF2DF010A428
:10595000ECEF2CF0BAC166F1BBC167F1BCC168F1D4
:10596000BDC169F1BEC16AF1BFC16BF1C0C16CF1CB
:10597000C1C16DF1C2C16EF1C3C16FF1C4C170F19B
:10598000C5C171F1C6C172F1C7C173F1C8C174F16B
:10599000C9C175F1CAC176F1CBC177F1CCC178F13B
:1059A000CDC179F1CEC17AF1CFC17BF1D0C17CF10B
:1059B000D1C17DF1D2C17EF1D3C17FF1D4C180F1DB
:1059C000D5C181F1D6C182F1D7C183F1D8C184F1AB
:1059D000D9C185F1F4EF2CF062C166F163C167F1C2
:1059E00064C168F165C169F1BAC186F1BBC187F1D3
:1059F000BCC188F1BDC189F14BC14FF14CC150F11F
:105A00004DC151F14EC152F157C159F158C15AF12E
:105A100007940FA02AEF2DF00101966717EF2DF0E4
:105A2000976717EF2DF0986717EF2DF099671BEF29
:105A30002DF02AEF2DF0AEEC2AF096C104F197C1BB
:105A400005F198C106F199C107F14AEC37F003BF9F
:105A500040EF30F0AEEC2AF00101000E046F000EB2
:105A6000056F010E066F000E076F7BEC37F011A07B
:105A70002AD011A228D0E8EC37F0296701D005D050
:105A800004012D0E826F5CEC0FF030C182F4040132
:105A9000300E82275CEC0FF031C182F40401300E2D
:105AA00082275CEC0FF032C182F40401300E8227B1
:105AB0005CEC0FF033C182F40401300E82275CEC01
:105AC0000FF066EC0FF012A8C5D012981AC01BF0A8
:105AD0001B3A1B42070E1B1600011B50000AD8B4CC
:105AE000F6EF2DF000011B50010AD8B482EF2DF023
:105AF00000011B50020AD8B480EF2DF028EF2EF0E1
:105B000028EF2EF045EC38F02AC001F12BC000F14F
:105B1000D89001330033D890013300330101630E74
:105B2000046F000E056F000E066F000E076F7BEC12
:105B300037F0280E046F000E056F000E066F000E82
:105B4000076F4AEC37F000C12DF045EC38F028C063
:105B500001F1019F019D29C000F10101A40E046F14
:105B6000000E056F000E066F000E076F7BEC37F01E
:105B700000C12CF000C104F101C105F102C106F120
:105B800003C107F1640E006F000E016F000E026F7B
:105B9000000E036F4AEC37F0050E046F000E056F20
:105BA000000E066F000E076F7BEC37F000C104F1AA
:105BB00001C105F102C106F103C107F145EC38F05E
:105BC0002DC000F14AEC37F000C12EF02EC0E8FFE6
:105BD000050F2D5C03E78A8428EF2EF02EC0E8FF26
:105BE0000A0F2D5C01E68A9428EF2EF000C124F103
:105BF00001C125F102C126F103C127F145EC38F0BE
:105C00004BEC38F01A501F0BE8CF00F10101640E85
:105C1000046F000E056F000E066F000E076F5BEC41
:105C200037F024C104F125C105F126C106F127C1D1
:105C300007F14AEC37F003BF02D08A9401D08A847E
:105C400024C100F125C101F126C102F127C103F1F0
:105C50007CEF30F000C124F101C125F102C126F131
:105C600003C127F110AE4DD0109E00C108F101C153
:105C700009F102C10AF103C10BF1E8EC37F030C1C0
:105C8000DAF131C1DBF132C1DCF133C1DDF108C140
:105C900000F109C101F10AC102F10BC103F10101D7
:105CA0006C0E046F070E056F000E066F000E076F77
:105CB0004AEC37F003BF04D00101550EDE6F1CD053
:105CC00008C100F109C101F10AC102F10BC103F1E0
:105CD0000101A40E046F060E056F000E066F000E84
:105CE000076F4AEC37F003BF04D001017F0EDE6F6F
:105CF00003D00101FF0EDE6F1C8E11AE40EF30F0BD
:105D0000119E24C100F125C101F126C102F127C174
:105D100003F111A005D011A203D00FB040EF30F075
:105D200010A49AEF2EF00401750E826F5CEC0FF058
:105D30009FEF2EF00401720E826F5CEC0FF00401F5
:105D40002C0E826F5CEC0FF0E8EC37F02967AEEFB9
:105D50002EF00401200E826FB1EF2EF004012D0E03
:105D6000826F5CEC0FF030C182F40401300E8227A8
:105D70005CEC0FF031C182F40401300E82275CEC40
:105D80000FF004012E0E826F5CEC0FF032C182F432
:105D90000401300E82275CEC0FF033C182F4040161
:105DA000300E82275CEC0FF004016D0E826F5CEC0C
:105DB0000FF004012C0E826F5CEC0FF04FC100F16C
:105DC00050C101F151C102F152C103F10101E8ECEE
:105DD00037F0ABEC35F00401480E826F5CEC0FF04D
:105DE00004017A0E826F5CEC0FF004012C0E826FBE
:105DF0005CEC0FF066C100F167C101F168C102F10E
:105E000069C103F10101E8EC37F0ABEC35F00401B6
:105E1000630E826F5CEC0FF004012C0E826F5CEC61
:105E20000FF066C100F167C101F168C102F169C1FB
:105E300003F101010A0E046F000E056F000E066FDC
:105E4000000E076F5BEC37F0000E046F120E056F4B
:105E5000000E066F000E076F7BEC37F0E8EC37F0B2
:105E60002AC182F40401300E82275CEC0FF02BC1B2
:105E700082F40401300E82275CEC0FF02CC182F416
:105E80000401300E82275CEC0FF02DC182F4040176
:105E9000300E82275CEC0FF02EC182F40401300E2C
:105EA00082275CEC0FF02FC182F40401300E8227B0
:105EB0005CEC0FF030C182F40401300E82275CEC00
:105EC0000FF004012E0E826F5CEC0FF031C182F4F2
:105ED0000401300E82275CEC0FF032C182F4040121
:105EE000300E82275CEC0FF033C182F40401300ED7
:105EF00082275CEC0FF00401730E826F5CEC0FF0F4
:105F000004012C0E826F5CEC0FF045EC38F059C1A7
:105F100000F15AC101F1A6EC31F013A2DFEF2FF02E
:105F200004012C0E826F5CEC0FF086C166F187C114
:105F300067F188C168F189C169F1AEEC2AF001010D
:105F4000000E046F000E056F010E066F000E076F46
:105F50007BEC37F0E8EC37F02967B4EF2FF0040161
:105F6000200E826FB7EF2FF004012D0E826F5CECD4
:105F70000FF030C182F40401300E82275CEC0FF088
:105F800031C182F40401300E82275CEC0FF0040171
:105F90002E0E826F5CEC0FF032C182F40401300EE1
:105FA00082275CEC0FF033C182F40401300E8227AB
:105FB0005CEC0FF004016D0E826F5CEC0FF013A42B
:105FC00006EF30F004012C0E826F5CEC0FF013AC86
:105FD000F4EF2FF00401500E826F5CEC0FF0139C75
:105FE0001398139A06EF30F013AE01EF30F004016E
:105FF000460E826F5CEC0FF0139E1398139A06EF17
:1060000030F00401530E826F5CEC0FF00FB20CEF16
:1060100030F00FA03EEF30F004012C0E826F5CECEC
:106020000FF0200EF86EF76AF66A04010900F5CF4A
:1060300082F45CEC0FF00900F5CF82F45CEC0FF019
:106040000900F5CF82F45CEC0FF00900F5CF82F483
:106050005CEC0FF00900F5CF82F45CEC0FF0090066
:10606000F5CF82F45CEC0FF00900F5CF82F45CEC24
:106070000FF00900F5CF82F45CEC0FF066EC0FF046
:106080000F90109E12987CEF30F00401630E826F27
:106090005CEC0FF004012C0E826F5CEC0FF082ECD4
:1060A00030F004012C0E826F5CEC0FF0F5EC30F058
:1060B00004012C0E826F5CEC0FF071EC31F00401E6
:1060C0002C0E826F5CEC0FF00101F80E006FCD0E0C
:1060D000016F660E026F030E036F97EC30F0040140
:1060E0002C0E826F5CEC0FF087EC31F066EC0FF059
:1060F0007CEF30F066EC0FF00301C26B079010925A
:106100008BEF33F0D8900E0ED4EC0BF0E8CF00F10B
:106110000F0ED4EC0BF0E8CF01F1100ED4EC0BF025
:10612000E8CF02F1110ED4EC0BF0E8CF03F101013E
:10613000000E046F000E056F010E066F000E076F54
:106140007BEC37F0E8EC37F02AC182F40401300E22
:1061500082275CEC0FF02BC182F40401300E822701
:106160005CEC0FF02CC182F40401300E82275CEC51
:106170000FF02DC182F40401300E82275CEC0FF089
:106180002EC182F40401300E82275CEC0FF02FC187
:1061900082F40401300E82275CEC0FF030C182F4EF
:1061A0000401300E82275CEC0FF031C182F404014F
:1061B000300E82275CEC0FF004012E0E826F5CEC37
:1061C0000FF032C182F40401300E82275CEC0FF034
:1061D00033C182F40401300E82275CEC0FF004011D
:1061E0006D0E826F5CEC0FF01200120ED4EC0BF00F
:1061F000E8CF00F1130ED4EC0BF0E8CF01F1140E50
:10620000D4EC0BF0E8CF02F1150ED4EC0BF0E8CF94
:1062100003F101010A0E046F000E056F000E066FF8
:10622000000E076F5BEC37F0000E046F120E056F67
:10623000000E066F000E076F7BEC37F0E8EC37F0CE
:106240002AC182F40401300E82275CEC0FF02BC1CE
:1062500082F40401300E82275CEC0FF02CC182F432
:106260000401300E82275CEC0FF02DC182F4040192
:10627000300E82275CEC0FF02EC182F40401300E48
:1062800082275CEC0FF02FC182F40401300E8227CC
:106290005CEC0FF030C182F40401300E82275CEC1C
:1062A0000FF004012E0E826F5CEC0FF031C182F40E
:1062B0000401300E82275CEC0FF032C182F404013D
:1062C000300E82275CEC0FF033C182F40401300EF3
:1062D00082275CEC0FF00401730E826F5CEC0FF010
:1062E00012000A0ED4EC0BF0E8CF00F10B0ED4EC48
:1062F0000BF0E8CF01F10C0ED4EC0BF0E8CF02F17B
:106300000D0ED4EC0BF0E8CF03F1A6EF31F0060E42
:10631000D4EC0BF0E8CF00F1070ED4EC0BF0E8CF93
:1063200001F1080ED4EC0BF0E8CF02F1090ED4EC29
:106330000BF0E8CF03F1A6EF31F0010145EC38F0A6
:10634000078457C100F158C101F107940101E80E1B
:10635000046F800E056F000E066F000E076F5BEC7A
:1063600037F0000E046F040E056F000E066F000E6E
:10637000076F7BEC37F0880E046F130E056F000E6D
:10638000066F000E076F4AEC37F00A0E046F000E1E
:10639000056F000E066F000E076F7BEC37F0E8EC20
:1063A00037F001012967DAEF31F00401200E826F26
:1063B000DDEF31F004012D0E826F5CEC0FF030C187
:1063C00082F40401300E82275CEC0FF031C182F4BC
:1063D0000401300E82275CEC0FF032C182F404011C
:1063E000300E82275CEC0FF004012E0E826F5CEC05
:1063F0000FF033C182F40401300E82275CEC0FF001
:106400000401430E826F5CEC0FF0120087C32AF187
:1064100088C32BF189C32CF18AC32DF18BC32EF1D4
:106420008CC32FF18DC330F18EC331F190C332F1A3
:1064300091C333F10101296B93EC38F00AEC38F089
:106440000101000E046F000E056F010E066F000EB5
:10645000076F5BEC37F00E0E0C6E00C10BF0BDEC5D
:106460000BF00F0E0C6E01C10BF0BDEC0BF0100E1B
:106470000C6E02C10BF0BDEC0BF0110E0C6E03C1E3
:106480000BF0BDEC0BF004017A0E826F5CEC0FF0A8
:1064900004012C0E826F5CEC0FF00401350E826F4C
:1064A0005CEC0FF004012C0E826F5CEC0FF082ECC0
:1064B00030F084EF2AF087C32AF188C32BF189C317
:1064C0002CF18AC32DF18BC32EF18CC32FF18DC318
:1064D00030F18EC331F190C332F191C333F1010138
:1064E000296B93EC38F00AEC38F0880E046F130E29
:1064F000056F000E066F000E076F4FEC37F0000EB1
:10650000046F040E056F000E066F000E076F5BEC44
:1065100037F00101E80E046F800E056F000E066F64
:10652000000E076F7BEC37F00A0E0C6E00C10BF00B
:10653000BDEC0BF00B0E0C6E01C10BF0BDEC0BF0C3
:106540000C0E0C6E02C10BF0BDEC0BF00D0E0C6EC0
:1065500003C10BF0BDEC0BF004017A0E826F5CEC12
:106560000FF004012C0E826F5CEC0FF00401360E6C
:10657000826F5CEC0FF004012C0E826F5CEC0FF06C
:1065800071EC31F084EF2AF087C32AF188C32BF134
:1065900089C32CF18AC32DF18BC32EF18CC32FF14B
:1065A0008DC330F18FC331F190C332F191C333F118
:1065B000010193EC38F00AEC38F0000E046F120E73
:1065C000056F000E066F000E076F5BEC37F00101E0
:1065D0000A0E046F000E056F000E066F000E076FA7
:1065E0007BEC37F0120E0C6E00C10BF0BDEC0BF023
:1065F000130E0C6E01C10BF0BDEC0BF0140E0C6E03
:1066000002C10BF0BDEC0BF0150E0C6E03C10BF0CC
:10661000BDEC0BF004017A0E826F5CEC0FF004010C
:106620002C0E826F5CEC0FF00401370E826F5CEC75
:106630000FF004012C0E826F5CEC0FF0F5EC30F0E3
:1066400084EF2AF087C32AF188C32BF189C32CF188
:106650008AC32DF18BC32EF18CC32FF18DC330F182
:106660008EC331F190C332F191C333F10101296B33
:1066700093EC38F00AEC38F0880E046F130E056FB7
:10668000000E066F000E076F4FEC37F0000E046F20
:10669000040E056F000E066F000E076F5BEC37F0FF
:1066A0000101E80E046F800E056F000E066F000EEC
:1066B000076F7BEC37F0060E0C6E00C10BF0BDECE3
:1066C0000BF0070E0C6E01C10BF0BDEC0BF0080EC9
:1066D0000C6E02C10BF0BDEC0BF0090E0C6E03C189
:1066E0000BF0BDEC0BF004017A0E826F5CEC0FF046
:1066F00004012C0E826F5CEC0FF00401380E826FE7
:106700005CEC0FF004012C0E826F5CEC0FF087EC58
:1067100031F084EF2AF007A8FEEF33F00101800E7C
:10672000006F1A0E016F060E026F000E036F4BC151
:1067300004F14CC105F14DC106F14EC107F14AEC1F
:1067400037F003BF44EF34F0A5EC35F04BC100F156
:106750004CC101F14DC102F14EC103F1078257EC6A
:1067600036F018C104F119C105F11AC106F11BC1B7
:1067700007F1F80E006FCD0E016F660E026F030E6B
:10678000036F4AEC37F00E0E0C6E00C10BF0BDEC3F
:106790000BF00F0E0C6E01C10BF0BDEC0BF0100EE8
:1067A0000C6E02C10BF0BDEC0BF0110E0C6E03C1B0
:1067B0000BF0BDEC0BF00784010145EC38F057C13C
:1067C00000F158C101F107940A0E0C6E00C10BF0E4
:1067D000BDEC0BF00B0E0C6E01C10BF0BDEC0BF021
:1067E0000C0E0C6E02C10BF0BDEC0BF00D0E0C6E1E
:1067F00003C10BF0BDEC0BF044EF34F007AA44EFFB
:1068000034F00784010145EC38F057C100F158C15C
:1068100001F10794060E0C6E00C10BF0BDEC0BF0FD
:10682000070E0C6E01C10BF0BDEC0BF0080E0C6EE8
:1068300002C10BF0BDEC0BF0090E0C6E03C10BF0A6
:10684000BDEC0BF0078462C100F163C101F164C1CA
:1068500002F165C103F10794120E0C6E00C10BF03A
:10686000BDEC0BF0130E0C6E01C10BF0BDEC0BF088
:10687000140E0C6E02C10BF0BDEC0BF0150E0C6E7D
:1068800003C10BF0BDEC0BF00798079A040180518F
:1068900081197F0B0DE09EA8FED714EE00F0815108
:1068A0007F0BE126E750812B0F01AD6E46EF34F0F0
:1068B00005012F51010A13E081AA80EF34F0050190
:1068C0002F51000A0AE00FB86FEF34F0050130676E
:1068D0006FEF34F00FB86FEF34F020EF42F081B873
:1068E00080EF34F094EC3AF080EF34F0602F80EFDA
:1068F00034F05FC560F50501010E306F3C0E316F5D
:106900009EEF0EF006013251385D3351D8A0010FD1
:10691000395D800BD8A491EF34F032C638F633C617
:1069200039F6120006013251365D3351D8A0010FFD
:10693000375D800BD8B4A1EF34F032C636F633C6DB
:1069400037F6120007841AC632F61BC633F61CC689
:1069500038F61DC639F682EC34F01EC632F61FC674
:1069600033F682EC34F020C632F621C633F682ECE0
:1069700034F01AC632F61BC633F61CC636F61DC6F0
:1069800037F692EC34F01EC632F61FC633F692ECA0
:1069900034F020C632F621C633F692EC34F038518A
:1069A000365F3951D8A03929375F45EC38F036C603
:1069B00000F137C601F151EC38F000C13AF601C1DF
:1069C0003BF622C632F623C633F624C638F625C671
:1069D00039F682EC34F026C632F627C633F682EC5E
:1069E00034F028C632F629C633F682EC34F022C6DB
:1069F00032F623C633F624C636F625C637F692ECB1
:106A000034F026C632F627C633F692EC34F028C6A8
:106A100032F629C633F692EC34F03851365F3951EC
:106A2000D8A03929375F45EC38F036C600F137C6B3
:106A300001F151EC38F000C13CF601C13DF62AC627
:106A400032F62BC633F62CC638F62DC639F682EC54
:106A500034F02EC632F62FC633F682EC34F030C650
:106A600032F631C633F682EC34F02AC632F62BC643
:106A700033F62CC636F62DC637F692EC34F02EC619
:106A800032F62FC633F692EC34F030C632F631C609
:106A900033F692EC34F03851365F3951D8A03929A9
:106AA000375F45EC38F036C600F137C601F151ECDE
:106AB00038F000C13EF601C13FF63AC632F63BC699
:106AC00033F63CC636F63DC637F692EC34F03EC699
:106AD00032F63FC633F692EC34F00794120018C138
:106AE00000F119C101F11AC102F11BC103F1000E3D
:106AF000046F000E056F010E066F000E076F7BEC32
:106B000037F029A19AEF35F02051D8B49AEF35F03B
:106B100018C100F119C101F11AC102F11BC103F141
:106B2000000E046F000E056F0A0E066F000E076F51
:106B30007BEC37F0120001010451001305510113E1
:106B4000065102130751031312000101186B196B50
:106B50001A6B1B6B12002AC182F40401300E8227CB
:106B60005CEC0FF02BC182F40401300E82275CEC48
:106B70000FF02CC182F40401300E82275CEC0FF080
:106B80002DC182F40401300E82275CEC0FF02EC17F
:106B900082F40401300E82275CEC0FF02FC182F4E6
:106BA0000401300E82275CEC0FF030C182F4040146
:106BB000300E82275CEC0FF031C182F40401300EFC
:106BC00082275CEC0FF032C182F40401300E822780
:106BD0005CEC0FF033C182F40401300E82275CECD0
:106BE0000FF012002FC182F40401300E82275CECFA
:106BF0000FF030C182F40401300E82275CEC0FF0FC
:106C000031C182F40401300E82275CEC0FF032C1F6
:106C100082F40401300E82275CEC0FF033C182F461
:106C20000401300E82275CEC0FF01200060E1E6E7F
:106C3000060E1F6E060E206E1E2E1CEF36F01F2E47
:106C40001CEF36F0202E1CEF36F08B84020E1E6EE9
:106C5000020E1F6E020E206E1E2E2CEF36F01F2E1F
:106C60002CEF36F0202E2CEF36F08B941200FF0E16
:106C70001F6E1FC020F0030E1E6E8B841E2E3DEF74
:106C800036F0030E1E6E202E3DEF36F08B941FC0A3
:106C900020F0030E1E6E1E2E4BEF36F0030E1E6EFE
:106CA000203E4BEF36F01F2E39EF36F01200010177
:106CB000005305E1015303E1025301E1002B1AECFB
:106CC00037F045EC38F03951006F3A51016F420E00
:106CD000046F4B0E056F000E066F000E076F5BEC26
:106CE00037F000C104F101C105F102C106F103C191
:106CF00007F118C100F119C101F11AC102F11BC15C
:106D000003F107B288EF36F04FEC37F08AEF36F038
:106D10004AEC37F000C118F101C119F102C11AF1B2
:106D200003C11BF1120045EC38F059C100F15AC102
:106D300001F1060ED4EC0BF0E8CF04F1070ED4EC11
:106D40000BF0E8CF05F1080ED4EC0BF0E8CF06F11C
:106D5000090ED4EC0BF0E8CF07F14AEC37F000C194
:106D600024F101C125F102C126F103C127F1290E49
:106D7000046F000E056F000E066F000E076F5BECD0
:106D800037F0EE0E046F430E056F000E066F000E17
:106D9000076F4FEC37F024C104F125C105F126C17E
:106DA00006F127C107F15BEC37F000C11CF101C10E
:106DB0001DF102C11EF103C11FF1120ED4EC0BF044
:106DC000E8CF04F1130ED4EC0BF0E8CF05F1140E6C
:106DD000D4EC0BF0E8CF06F1150ED4EC0BF0E8CFB5
:106DE00007F10D0E006F000E016F000E026F000E16
:106DF000036F5BEC37F0180E046F000E056F000E8A
:106E0000066F000E076F7BEC37F01CC104F11DC14B
:106E100005F11EC106F11FC107F14FEC37F06A0EF4
:106E2000046F2A0E056F000E066F000E076F4AEC06
:106E300037F01200BF0EFA6E200E3A6F396BD89001
:106E40000037013702370337D8B02BEF37F03A2F2E
:106E500020EF37F039073A070353D8B41200033153
:106E6000070B80093F6F03390F0B010F396F80EC5F
:106E70005FF0406F390580EC5FF0405D405F396B3B
:106E80003F33D8B0392739333FA940EF37F040516D
:106E90003927120001016AEC38F0D8B01200010164
:106EA00003510719346F2DEC38F0D89007510319AE
:106EB00034AF800F12000101346B51EC38F0D8A0D0
:106EC00067EC38F0D8B012003CEC38F045EC38F004
:106ED0001F0E366F7DEC38F00B35D8B02DEC38F046
:106EE000D8A00335D8B01200362F6AEF37F034B18E
:106EF00054EC38F012000101346B045105110611F5
:106F000007110008D8A051EC38F0D8A067EC38F091
:106F1000D8B01200086B096B0A6B0B6B7DEC38F074
:106F20001F0E366F7DEC38F007510B5DD8A4A5EF2E
:106F300037F006510A5DD8A4A5EF37F00551095D79
:106F4000D8A4A5EF37F00451085DD8A0B8EF37F00A
:106F50000451085F0551D8A0053D095F0651D8A02E
:106F6000063D0A5F0751D8A0073D0B5FD89000810E
:106F7000362F92EF37F034B154EC38F0346B51ECDB
:106F800038F0D89081EC38F007510B5DD8A4D5EFDC
:106F900037F006510A5DD8A4D5EF37F00551095DE9
:106FA000D8A4D5EF37F00451085DD8A0E4EF37F04E
:106FB000003FE4EF37F0013FE4EF37F0023FE4EF4A
:106FC00037F0032BD8B4120034B154EC38F012006F
:106FD0000101346B51EC38F0D8B0120086EC38F077
:106FE000200E366F003701370237033711EE33F0CA
:106FF0000A0E376FE7360A0EE75CD8B0E76EE55247
:10700000372FFAEF37F0362FF2EF37F034B129810E
:10701000D890120001010A0E346F200E366F11EE67
:1070200029F03451376F0A0ED890E652D8B0E726CF
:10703000E732372F15EF38F00333023301330033D3
:10704000362F0FEF38F0E750FF0FD8A00335D8B038
:10705000120029B154EC38F01200045100270551F8
:10706000D8B0053D01270651D8B0063D022707518B
:10707000D8B0073D032712000051086F0151096F76
:1070800002510A6F03510B6F12000101006B016B7B
:10709000026B036B12000101046B056B066B076B3F
:1070A00012000335D8A012000351800B001F011FEE
:1070B000021F031F003F64EF38F0013F64EF38F018
:1070C000023F64EF38F0032B342B03251200073501
:1070D000D8A012000751800B041F051F061F071FB1
:1070E000043F7AEF38F0053F7AEF38F0063F7AEF49
:1070F00038F0072B342B07251200003701370237F1
:107100000337083709370A370B3712000101296B9B
:107110002A6B2B6B2C6B2D6B2E6B2F6B306B316BAB
:10712000326B336B120001012A510F0B2A6F2B5166
:107130000F0B2B6F2C510F0B2C6F2D510F0B2D6F35
:107140002E510F0B2E6F2F510F0B2F6F30510F0B36
:10715000306F31510F0B316F32510F0B326F335192
:107160000F0B336F1200899C000EC76E200EC66E87
:107170009E96C69EC50EC96EFF0E9EB602D0E82E24
:10718000FCD79E96C69E000EC96EFF0E9EB602D01C
:10719000E82EFCD7C9CF00F69E96C69E000EC96E9B
:1071A000FF0E9EB602D0E82EFCD7C9CF01F6898C1F
:1071B0001200000EC76E200EC66E899C9E96C69E5B
:1071C000C80EC96EFF0E9EB602D0E82EFCD79E9662
:1071D000C69E000EC96EFF0E9EB602D0E82EFCD7EA
:1071E000C9CF02F69E96C69E000EC96EFF0E9EB6D1
:1071F00002D0E82EFCD7C9CF03F69E96C69E000E9D
:10720000C96EFF0E9EB602D0E82EFCD7C9CF0AF693
:107210009E96C69E000EC96EFF0E9EB602D0E82E48
:10722000FCD7C9CF0BF69E96C69E000EC96EFF0E08
:107230009EB602D0E82EFCD7C9CF12F69E96C69E07
:10724000000EC96EFF0E9EB602D0E82EFCD7C9CF45
:1072500013F6898C1200000EC76E200EC66E899C34
:107260009E96C69EE80EC96EFF0E9EB602D0E82E10
:10727000FCD79E96C69E000EC96EFF0E9EB602D02B
:10728000E82EFCD7C9CF1AF69E96C69E000EC96E90
:10729000FF0E9EB602D0E82EFCD7C9CF1BF69E96F5
:1072A000C69E000EC96EFF0E9EB602D0E82EFCD719
:1072B000C9CF22F69E96C69E000EC96EFF0E9EB6E0
:1072C00002D0E82EFCD7C9CF23F69E96C69E000EAC
:1072D000C96EFF0E9EB602D0E82EFCD7C9CF2AF6A3
:1072E0009E96C69E000EC96EFF0E9EB602D0E82E78
:1072F000FCD7C9CF2BF6898C1200000EC76E200E6A
:10730000C66E899C9E96C69E240EC96EFF0E9EB6C2
:1073100002D0E82EFCD79E96C69EE40EC96EFF0EE4
:107320009EB602D0E82EFCD7898C899C9E96C69E7C
:10733000200EC96EFF0E9EB602D0E82EFCD79E9698
:10734000C69E5F0EC96EFF0E9EB602D0E82EFCD719
:10735000898C899C9E96C69E210EC96EFF0E9EB694
:1073600002D0E82EFCD79E96C69EC00EC96EFF0EB8
:107370009EB602D0E82EFCD7898C899C9E96C69E2C
:10738000260EC96EFF0E9EB602D0E82EFCD79E9642
:10739000C69E000EC96EFF0E9EB602D0E82EFCD728
:1073A000898C120010A806D08994000EC76E220E98
:1073B000C66E05D08984000EC76E220EC66E050EFD
:1073C000E82EFED7120010A802D0898401D089943B
:1073D000050EE82EFED71200D2EC39F09E96C69E1E
:1073E000000EC96EFF0E9EB602D0E82EFCD79E9608
:1073F000C69E000EC96EFF0E9EB602D0E82EFCD7C8
:10740000C9CFAFF59E96C69E000EC96EFF0E9EB602
:1074100002D0E82EFCD7C9CFB0F59E96C69E000ECE
:10742000C96EFF0E9EB602D0E82EFCD7C9CFB1F5CB
:107430009E96C69E000EC96EFF0E9EB602D0E82E26
:10744000FCD7C9CFB2F59E96C69E000EC96EFF0E40
:107450009EB602D0E82EFCD7C9CFB3F59E96C69E45
:10746000000EC96EFF0E9EB602D0E82EFCD7C9CF23
:10747000B4F59E96C69E000EC96EFF0E9EB602D053
:10748000E82EFCD7C9CFB5F5E3EC39F01200D2EC09
:1074900039F09E96C69E800EC96EFF0E9EB602D033
:1074A000E82EFCD79E96C69EAFC5C9FFFF0E9EB6BE
:1074B00002D0E82EFCD79E96C69EB0C5C9FFFF0E2F
:1074C0009EB602D0E82EFCD79E96C69EB1C5C9FFD7
:1074D000FF0E9EB602D0E82EFCD79E96C69EB2C581
:1074E000C9FFFF0E9EB602D0E82EFCD79E96C69E20
:1074F000B3C5C9FFFF0E9EB602D0E82EFCD79E96FC
:10750000C69EB4C5C9FFFF0E9EB602D0E82EFCD7BA
:107510009E96C69EB5C5C9FFFF0E9EB602D0E82E48
:10752000FCD7E3EC39F01200D2EC39F09E96C69EFF
:10753000070EC96EFF0E9EB602D0E82EFCD79E96AF
:10754000C69E000EC96EFF0E9EB602D0E82EFCD776
:10755000C9CFAFF59E96C69E000EC96EFF0E9EB6B1
:1075600002D0E82EFCD7C9CFB0F59E96C69E000E7D
:10757000C96EFF0E9EB602D0E82EFCD7C9CFB1F57A
:107580009E96C69E000EC96EFF0E9EB602D0E82ED5
:10759000FCD7C9CFB2F5E3EC39F0D2EC39F09E96C6
:1075A000C69E22C0C9FFFF0E9EB602D0E82EFCD7B1
:1075B0009E96C69E000EC96EFF0E9EB602D0E82EA5
:1075C000FCD7C9CFB6F5E3EC39F01200D2EC39F0B4
:1075D0009E96C69E870EC96EFF0E9EB602D0E82EFE
:1075E000FCD79E96C69EAFC5C9FFFF0E9EB602D0C1
:1075F000E82EFCD79E96C69EB0C5C9FFFF0E9EB66C
:1076000002D0E82EFCD79E96C69EB1C5C9FFFF0EDC
:107610009EB602D0E82EFCD79E96C69EB2C5C9FF84
:10762000FF0E9EB602D0E82EFCD7E3EC39F0D2EC88
:1076300039F09E96C69E23C0C9FFFF0E9EB602D0AB
:10764000E82EFCD79E96C69EB6C5C9FFFF0E9EB615
:1076500002D0E82EFCD7E3EC39F01200D2EC39F07E
:107660009E96C69E870EC96EFF0E9EB602D0E82E6D
:10767000FCD79E96C69E000EC96EFF0E9EB602D027
:10768000E82EFCD79E96C69E800EC96EFF0E9EB653
:1076900002D0E82EFCD79E96C69E800EC96EFF0EC5
:1076A0009EB602D0E82EFCD79E96C69E800EC96E6E
:1076B000FF0E9EB602D0E82EFCD7E3EC39F01200A4
:1076C000D2EC39F09E96C69E870EC96EFF0E9EB60E
:1076D00002D0E82EFCD79E96C69E000EC96EFF0E05
:1076E0009EB602D0E82EFCD79E96C69E000EC96EAE
:1076F000FF0E9EB602D0E82EFCD79E96C69E800E48
:10770000C96EFF0E9EB602D0E82EFCD79E96C69E8E
:10771000800EC96EFF0E9EB602D0E82EFCD7E3ECB9
:1077200039F0120010A817D0D2EC39F09E96C69E00
:107730008F0EC96EFF0E9EB602D0E82EFCD79E9625
:10774000C69E000EC96EFF0E9EB602D0E82EFCD774
:10775000E3EC39F0120094EC3AF0120010A82DD0AE
:10776000D2EC39F09E96C69E23C0C9FFFF0E9EB68E
:1077700002D0E82EFCD79E96C69E450EC96EFF0E1F
:107780009EB602D0E82EFCD7E3EC39F0D2EC39F00B
:107790009E96C69E8F0EC96EFF0E9EB602D0E82E34
:1077A000FCD79E96C69E000EC96EFF0E9EB602D0F6
:1077B000E82EFCD7E3EC39F01200D2EC39F09E96BB
:1077C000C69E23C0C9FFFF0E9EB602D0E82EFCD78E
:1077D0009E96C69E010EC96EFF0E9EB602D0E82E82
:1077E000FCD7E3EC39F0D2EC39F09E96C69E910EB0
:1077F000C96EFF0E9EB602D0E82EFCD79E96C69E9E
:10780000A50EC96EFF0E9EB602D0E82EFCD7E3ECA3
:1078100039F01200D2EC39F09E96C69E23C0C9FF03
:10782000FF0E9EB602D0E82EFCD79E96C69E810E15
:10783000C96EFF0E9EB602D0E82EFCD7E3EC39F0FD
:107840001200D2EC39F09E96C69E23C0C9FFFF0EEF
:107850009EB602D0E82EFCD79E96C69E010EC96E3B
:10786000FF0E9EB602D0E82EFCD7E3EC39F01200F2
:10787000D2EC39F09E96C69E910EC96EFF0E9EB652
:1078800002D0E82EFCD79E96C69EA50EC96EFF0EAE
:107890009EB602D0E82EFCD7E3EC39F01200D2EC11
:1078A00039F09E96C69E910EC96EFF0E9EB602D00E
:1078B000E82EFCD79E96C69E000EC96EFF0E9EB6A1
:1078C00002D0E82EFCD7E3EC39F012000501256B5D
:1078D000266B276B286B899A400EC76E200EC66EEA
:1078E0009E96C69E030EC96EFF0E9EB602D0E82E6F
:1078F000FCD79E96C69E27C5C9FFFF0E9EB602D036
:10790000E82EFCD79E96C69E26C5C9FFFF0E9EB6E2
:1079100002D0E82EFCD79E96C69E25C5C9FFFF0E55
:107920009EB602D0E82EFCD79E96C69EC952FF0E88
:107930009EB602D0E82EFCD7898A0F01C950FF0AF3
:1079400001E1120005012E51130A05E005012E5137
:10795000170A0CE012000501E00E256FFF0E266FDE
:107960000F0E276F000E286FBFEF3CF00501E00EF1
:10797000256FFF0E266FFF0E276F000E286F899A66
:10798000400EC76E200EC66E9E96C69E030EC96E32
:10799000FF0E9EB602D0E82EFCD79E96C69E27C547
:1079A000C9FFFF0E9EB602D0E82EFCD79E96C69E5B
:1079B00026C5C9FFFF0E9EB602D0E82EFCD79E96C4
:1079C000C69E25C5C9FFFF0E9EB602D0E82EFCD785
:1079D0009E96C69EC952FF0E9EB602D0E82EFCD7D8
:1079E000898A0F01C950FF0A1DE005012E51130AB3
:1079F00005E005012E51170A0BE012000501000EEB
:107A0000256F000E266F100E276F000E286F1200D4
:107A10000501000E256F000E266F000E276F010E68
:107A2000286F12000501256B266B276B286B05015B
:107A30002E51130A05E005012E51170A0CE0120021
:107A40000501000E216F000E226F080E236F000E3D
:107A5000246F34EF3DF00501000E216F000E226F00
:107A6000800E236F000E246F21C500F122C501F1A5
:107A700023C502F124C503F125C504F126C505F18E
:107A800027C506F128C507F19BEC35F000C125F5A7
:107A900001C126F502C127F503C128F5899A400ED8
:107AA000C76E200EC66E9E96C69E030EC96EFF0E52
:107AB0009EB602D0E82EFCD79E96C69E27C5C9FF6B
:107AC000FF0E9EB602D0E82EFCD79E96C69E26C517
:107AD000C9FFFF0E9EB602D0E82EFCD79E96C69E2A
:107AE00025C5C9FFFF0E9EB602D0E82EFCD79E9694
:107AF000C69EC952FF0E9EB602D0E82EFCD7898AD8
:107B0000C950FF0A08E104C125F505C126F506C1E3
:107B100027F507C128F5D8900501243323332233F4
:107B200021332151E00B216F21679EEF3DF0226749
:107B30009EEF3DF023679EEF3DF0246734EF3DF06C
:107B40000501200E2527E86A2623E86A2723E86A2C
:107B500028231200E86A05012E51130A06E00501E8
:107B60002E51170A0BE0020E120005012851000ADF
:107B700003E12751F00B07E0010E12000501285127
:107B8000000A01E0010E120029C500F12AC501F129
:107B90002BC502F12CC503F125C504F126C505F15D
:107BA00027C506F128C507F14AEC37F003BF1200DC
:107BB000AAEC3DF0D8A43CEF3EF0899A400EC76E87
:107BC000200EC66E9E96C69E060EC96EFF0E9EB60F
:107BD00002D0E82EFCD7898A899A9E96C69E020E0C
:107BE000C96EFF0E9EB602D0E82EFCD79E96C69EAA
:107BF00027C5C9FFFF0E9EB602D0E82EFCD79E9681
:107C0000C69E26C5C9FFFF0E9EB602D0E82EFCD741
:107C10009E96C69E25C5C9FFFF0E9EB602D0E82ED1
:107C2000FCD79E96C69E000EC96EFF0E9EB602D071
:107C3000E82EFCD7898A899A9E96C69E050EC96E43
:107C4000FF0E9EB602D0E82EFCD79E96C69EC95265
:107C5000FF0E9EB602D0E82EFCD7C9B025EF3EF04D
:107C6000898A0501200E2527E86A2623E86A27234A
:107C7000E86A2823C4EF3DF01200899A400EC76ECF
:107C8000200EC66E9E96C69E060EC96EFF0E9EB64E
:107C900002D0E82EFCD7898A899A9E96C69EC70E86
:107CA000C96EFF0E9EB602D0E82EFCD7898A050168
:107CB000256B266B276B286B1200899A400EC76EC6
:107CC000200EC66E9E96C69E050EC96EFF0E9EB60F
:107CD00002D0E82EFCD79E96C69EC952FF0E9EB6D5
:107CE00002D0E82EFCD7C9CF37F5898A1200899ACD
:107CF000400EC76E200EC66E9E96C69EB90EC96E09
:107D0000FF0E9EB602D0E82EFCD7898A1200899A0F
:107D1000400EC76E200EC66E9E96C69EAB0EC96EF6
:107D2000FF0E9EB602D0E82EFCD7898AFF0EE82E01
:107D3000FED71200AAEC3DF0D8A41200899A400E9A
:107D4000C76E200EC66E9E96C69E030EC96EFF0EAF
:107D50009EB602D0E82EFCD79E96C69E27C5C9FFC8
:107D6000FF0E9EB602D0E82EFCD79E96C69E26C574
:107D7000C9FFFF0E9EB602D0E82EFCD79E96C69E87
:107D800025C5C9FFFF0E9EB602D0E82EFCD79E96F1
:107D9000C69EC952FF0E9EB602D0E82EFCD7898A35
:107DA0000F01C950FF0AD8A493EF41F00501FE0E60
:107DB000376F30A03799ECEC39F0AFC538F5B0C566
:107DC00039F5B1C53AF5B2C53BF5B3C53CF5B4C517
:107DD0003DF5B5C53EF50784BAC166F1BBC167F193
:107DE000BCC168F1BDC169F14BC14FF14CC150F14B
:107DF0004DC151F14EC152F157C159F158C15AF11B
:107E0000AEEC2AF000C13FF501C140F502C141F5D9
:107E100003C142F50501616715EF3FF0626715EF99
:107E20003FF0636715EF3FF0646719EF3FF026EF0F
:107E30003FF061C504F162C505F163C506F164C593
:107E400007F14AEC37F003BF93EF41F059C143F516
:107E50005AC144F5B9C545F5BAC546F5A2EC34F0AA
:107E600036C649F537C64AF5060140673FEF3FF091
:107E700041673FEF3FF042673FEF3FF0436743EF1B
:107E80003FF054EF3FF045EC38F04BEC38F036C69D
:107E900000F137C601F140C604F141C605F14AECD4
:107EA00037F003AF93EF41F00101036B026B1AC689
:107EB00000F11BC601F101AF62EF3FF0FF0E026F50
:107EC000FF0E036F0101076B066B1CC604F11DC694
:107ED00005F105AF70EF3FF0FF0E066FFF0E076F65
:107EE0004FEC37F00101076B066B1EC604F11FC68D
:107EF00005F105AF80EF3FF0FF0E066FFF0E076F35
:107F00004FEC37F00101076B066B20C604F121C668
:107F100005F105AF90EF3FF0FF0E066FFF0E076F04
:107F20004FEC37F0D89001010333023301330033B3
:107F3000D8900101033302330133003300C14BF504
:107F400001C14CF50101036B026B22C600F123C68F
:107F500001F101AFB0EF3FF0FF0E026FFF0E036FB4
:107F60000101076B066B24C604F125C605F105AFB8
:107F7000BEEF3FF0FF0E066FFF0E076F4FEC37F0BE
:107F80000101076B066B26C604F127C605F105AF94
:107F9000CEEF3FF0FF0E066FFF0E076F4FEC37F08E
:107FA0000101076B066B28C604F129C605F105AF70
:107FB000DEEF3FF0FF0E066FFF0E076F4FEC37F05E
:107FC000D89001010333023301330033D89001010B
:107FD000033302330133003300C14DF501C14EF5C7
:107FE0000101036B026B2AC600F12BC601F101AF40
:107FF000FEEF3FF0FF0E026FFF0E036F0101076BF4
:10800000066B2CC604F12DC605F105AF0CEF40F050
:10801000FF0E066FFF0E076F4FEC37F00101076B85
:10802000066B2EC604F12FC605F105AF1CEF40F01C
:10803000FF0E066FFF0E076F4FEC37F00101076B65
:10804000066B30C604F131C605F105AF2CEF40F0E8
:10805000FF0E066FFF0E076F4FEC37F0D89001014F
:108060000333023301330033D89001010333023369
:108070000133003300C14FF501C150F50101036B1D
:10808000026B02C600F103C601F101AF4CEF40F0F4
:10809000FF0E026FFF0E036F0101076B066B04C634
:1080A00004F105C605F105AF5AEF40F0FF0E066F6B
:1080B000FF0E076F4FEC37F00101076B066B06C62A
:1080C00004F107C605F105AF6AEF40F0FF0E066F39
:1080D000FF0E076F4FEC37F00101076B066B08C608
:1080E00004F109C605F105AF7AEF40F0FF0E066F07
:1080F000FF0E076F4FEC37F0D890010103330233C6
:1081000001330033D89001010333023301330033CC
:1081100000C151F501C152F50101036B026B0AC6A2
:1081200000F10BC601F101AF9AEF40F0FF0E026FB4
:10813000FF0E036F0101076B066B0CC604F10DC641
:1081400005F105AFA8EF40F0FF0E066FFF0E076FB9
:108150004FEC37F00101076B066B0EC604F10FC63A
:1081600005F105AFB8EF40F0FF0E066FFF0E076F89
:108170004FEC37F00101076B066B10C604F111C616
:1081800005F105AFC8EF40F0FF0E066FFF0E076F59
:108190004FEC37F0D8900101033302330133003341
:1081A000D8900101033302330133003300C153F58A
:1081B00001C154F50101036B026B12C600F113C635
:1081C00001F101AFE8EF40F0FF0E026FFF0E036F09
:1081D0000101076B066B14C604F115C605F105AF66
:1081E000F6EF40F0FF0E066FFF0E076F4FEC37F013
:1081F0000101076B066B16C604F117C605F105AF42
:1082000006EF41F0FF0E066FFF0E076F4FEC37F0E1
:108210000101076B066B18C604F119C605F105AF1D
:1082200016EF41F0FF0E066FFF0E076F4FEC37F0B1
:10823000D89001010333023301330033D890010198
:10824000033302330133003300C155F501C156F544
:1082500007940501210E326F899A400EC76E200ED9
:10826000C66E9E96C69E060EC96EFF0E9EB602D0C4
:10827000E82EFCD7898A899A9E96C69E020EC96E00
:10828000FF0E9EB602D0E82EFCD79E96C69E27C54E
:10829000C9FFFF0E9EB602D0E82EFCD79E96C69E62
:1082A00026C5C9FFFF0E9EB602D0E82EFCD79E96CB
:1082B000C69E25C5C9FFFF0E9EB602D0E82EFCD78C
:1082C00025EE37F0322F02D071EF41F09E96C69E18
:1082D000DECFC9FFFF0E9EB602D0E82EFCD762EFBC
:1082E00041F0898A899A9E96C69E050EC96EFF0E38
:1082F0009EB602D0E82EFCD79E96C69EC952FF0EAF
:108300009EB602D0E82EFCD7C9B07CEF41F0898A36
:108310000501200E2527E86A2623E86A2723E86A54
:10832000282316EC36F0120021C500F122C501F118
:1083300023C502F124C503F1899A400EC76E200EB1
:10834000C66E9E96C69E0B0EC96EFF0E9EB602D0DE
:10835000E82EFCD79E96C69E02C1C9FFFF0E9EB6B0
:1083600002D0E82EFCD79E96C69E01C1C9FFFF0E23
:108370009EB602D0E82EFCD79E96C69E00C1C9FFCD
:10838000FF0E9EB602D0E82EFCD79E96C69EC9521E
:10839000FF0E9EB602D0E82EFCD725EE37F0050181
:1083A000200E326F9E96C69EC952FF0E9EB602D018
:1083B000E82EFCD7C9CFDEFF322FD2EF41F0898AF9
:1083C0001200899A400EC76E200EC66E9E96C69EFB
:1083D000900EC96EFF0E9EB602D0E82EFCD79E9678
:1083E000C69E000EC96EFF0E9EB602D0E82EFCD7C8
:1083F0009E96C69E000EC96EFF0E9EB602D0E82E57
:10840000FCD79E96C69E000EC96EFF0E9EB602D089
:10841000E82EFCD79E96C69EC952FF0E9EB602D08D
:10842000E82EFCD7C9CF2DF59E96C69EC952FF0EE9
:108430009EB602D0E82EFCD7C9CF2EF5898A12004D
:1084400016EC36F0B9C5E8FFD70802E316EC36F0B3
:10845000B9C5E8FFC80802E316EC36F0B9C5E8FF75
:10846000B90802E316EC36F0B9C5E8FFAA0802E342
:1084700016EC36F0B9C5E8FF9B0802E316EC36F0BF
:1084800077EC3EF0F29CF29E8B94C69AC290898C57
:108490009482948C720ED36ED3A4FED789968A9060
:1084A0009390F29AF2949D909E909D929E92F29853
:1084B000F29292EC3BF0FF0EE8CF00F0E82EFED7F0
:1084C000002EFCD7F290F286815081A86AEF42F02C
:1084D000F29E0300700ED36EF296F290010E306E93
:0A84E000038037EC36F009EF0CF0D2
:10BF0000E844F926000C160C2B0C3F0C520C640C68
:10BF1000760C860C960CA50CB30CC10CCF0CDC0C6B
:06BF2000E80CF40C000C1B
:00000001FF
